:0200000480007A
:10000000B72F0000938F0F8073900F306F00400365
:100010001300000013000000130000001300000094
:100020001300000013000000130000001300000084
:100030001300000013000000130000001300000074
:100040009702000093824211739052309300000097
:10005000130100009301000013020000930200004E
:100060001303000093030000130400009304000036
:10007000130500009305000013060000930600001E
:100080001307000093070000130800009308000006
:100090001309000093090000130A0000930A0000EE
:1000A000130B0000930B0000130C0000930C0000D6
:1000B000130D0000930D0000130E0000930E0000BE
:1000C000130F0000930F000097110200938141BDB0
:1000D000170502001305053F979503009385857169
:1000E00013060000EF00001A170502001305853AF9
:1000F000970502009385853A13060000EF008018EB
:1001000017A503001305456F97B503009385856E0A
:1001100037B6ABAB1306B6BAEF00C01617B1030083
:100120001301816DEF70803E9392120093D2120002
:100130009382D2FF638A02008322010013014100EF
:100140006F0000177300203083220100130141006B
:10015000730020301301C1FF23205100F32220340B
:10016000E3C402FC8322010013014100130141F8A2
:1001700023221100232421002326310023284100BB
:10018000232A5100232C6100232E71002320810299
:10019000232291022324A1022326B1022328C10293
:1001A000232AD102232CE102232EF1022320010570
:1001B0002322110523242105232631052328410567
:1001C000232A5105232C6105232E71052320810745
:1001D000232291072324A1072326B1072328C1073F
:1001E000232AD107232CE107232EF107732520347E
:1001F000F3251034130601006F000000731015344E
:1002000083204100032181008321C10003220101D9
:1002100083224101032381018323C10103240102BD
:1002200083244102032581028325C10203260103A1
:1002300083264103032781038327C1030328010485
:1002400083284104032981048329C104032A010569
:10025000832A4105032B8105832BC105032C01064D
:10026000832C4106032D8106832DC106032E010731
:10027000832E4107032F8107832FC1071301C10775
:10028000730020302320C5006376B50013054500B8
:100290006FF05FFF678000000000000000000000BA
:1002A000000000000000000000000000000000004E
:1002B000130101F8232011002322210023243100FF
:1002C0002326410023285100232A6100232C71009A
:1002D000232E8100232091022322A1022324B10294
:1002E0002326C1022328D102232AE102232CF10272
:1002F000232E010323201105232221052324310568
:100300002326410523285105232A6105232C710545
:10031000232E8105232091072322A1072324B1073F
:100320002326C1072328D107232AE107232CF1071D
:100330009702020083A2021623A02200F3221034A7
:10034000232E5106EF00804617010200032181147D
:10035000032101008322C10773901234B7220000E9
:100360009382028873A00230832001000322C1001F
:100370008322010103234101832381010324C1015D
:100380008324010203254102832581020326C10241
:100390008326010303274103832781030328C10325
:1003A000832801040329410483298104032AC10409
:1003B000832A0105032B4105832B8105032CC105ED
:1003C000832C0106032D4106832D8106032EC106D1
:1003D000832E0107032F4107832F81071301010893
:1003E00073002030970202009382C20D23A01200F6
:1003F00023A2220023A4320023A6420023A85200F5
:1004000023AA620023AC720023AE820023A09202D2
:1004100023A2A20223A4B20223A6C20223A8D202CC
:1004200023AAE20223ACF20223AE020323A01205A8
:1004300023A2220523A4320523A6420523A85205A0
:1004400023AA620523AC720523AE820523A092077E
:1004500023A2A20723A4B20723A6C20723A8D20778
:1004600023AAE20723ACF207EF6010731701020022
:1004700003214102032101008322C107739012343A
:10048000B72200009382028873A00230832001000B
:100490000322C1008322010103234101832381013F
:1004A0000324C10183240102032541028325810223
:1004B0000326C10283260103032741038327810307
:1004C0000328C103832801040329410483298104EB
:1004D000032AC104832A0105032B4105832B8105CF
:1004E000032CC105832C0106032D4106832D8106B3
:1004F000032EC106832E0107032F4107832F810797
:10050000130101087300203097020200938282FBDE
:1005100083A0020003A1420083A1820003A2C200C3
:1005200083A2020103A3420183A3820103A4C201A7
:1005300083A4020203A5420283A5820203A6C2028B
:1005400083A6020303A7420383A7820303A8C2036F
:1005500083A8020403A9420483A9820403AAC20453
:1005600083AA020503AB420583AB820503ACC20537
:1005700083AC020603AD420683AD820603AEC2061B
:1005800083AE020703AFC20983AF82076780000012
:1005900073700430130101F823201100232221007D
:1005A000232431002326410023285100232A6100FF
:1005B000232C7100232E8100232091022322A102EB
:1005C0002324B1022326C1022328D102232AE102D7
:1005D000232CF102232E01032320110523222105C0
:1005E000232431052326410523285105232A6105AB
:1005F000232C7105232E8105232091072322A10797
:100600002324B1072326C1072328D107232AE10782
:10061000232CF1079702020083A2C2E723A0220045
:10062000232E1106EF20D05817010200032181E686
:10063000032101008322C10773901234B722000006
:100640009382028873A00230832001000322C1003C
:100650008322010103234101832381010324C1017A
:100660008324010203254102832581020326C1025E
:100670008326010303274103832781030328C10342
:10068000832801040329410483298104032AC10426
:10069000832A0105032B4105832B8105032CC1050A
:1006A000832C0106032D4106832D8106032EC106EE
:1006B000832E0107032F4107832F810713010108B0
:1006C0007300203097070200938787DD03A7070098
:1006D0009307F0FF6306F700737004306F000000AB
:1006E000737004306F000000130101FF2326A10086
:1006F0008327C100739047301300000013010101EC
:1007000067800000130101FFF32740302326F1002A
:1007100073F043308327C1001385070013010101E3
:1007200067800000130101FF2326A1002324B100EC
:100730002322C1008327C1009387C7FF2326F1002E
:10074000032781008327C10023A0E7008327C1007E
:10075000938787FA2326F100032741008327C100EE
:1007600023A0E7008327C100938787FE2326F1009B
:1007700093870100138707008327C10023A0E700A8
:100780008327C100938747FF2326F1001707000046
:10079000130787F38327C10023A0E7008327C10045
:1007A000138507001301010167800000130101FF99
:1007B00023261100EF60D033EF20101693070500B9
:1007C00063840700EF20D03E130000008320C100A7
:1007D0001301010167800000130101FF2326A1001E
:1007E0008327C100138787008327C10023A2E70066
:1007F0008327C1001307F0FF23A4E7008327C1006C
:10080000138787008327C10023A6E7008327C10041
:10081000138787008327C10023A8E7008327C1002F
:1008200023A00700130000001301010167800000EE
:10083000130101FF2326A1008327C10023A807007D
:10084000130000001301010167800000130101FE85
:100850002326A1002324B1008327C10083A74700DA
:10086000232EF100832781000327C10123A2E70083
:100870008327C10103A787008327810023A4E70002
:100880008327C10183A787000327810023A2E700F4
:100890008327C1010327810023A4E7008327810068
:1008A0000327C10023A8E7008327C10083A707000F
:1008B000138717008327C10023A0E700130000005F
:1008C0001301010267800000130101FE2326A1002D
:1008D0002324B1008327810083A70700232CF10084
:1008E000032781019307F0FF631AF7008327C100F4
:1008F00083A70701232EF1006F0040038327C10067
:1009000093878700232EF1006F0000018327C10128
:1009100083A74700232EF1008327C10183A7470047
:1009200083A7070003278101E372F7FE8327C10134
:1009300003A747008327810023A2E70083278100C4
:1009400083A747000327810023A4E70083278100B2
:100950000327C10123A4E7008327C10103278100E6
:1009600023A2E700832781000327C10023A8E70013
:100970008327C10083A70700138717008327C100BF
:1009800023A0E700130000001301010267800000AC
:10099000130101FE2326A1008327C10083A70701BD
:1009A000232EF1008327C10083A747000327C1003E
:1009B0000327870023A4E7008327C10083A78700BC
:1009C0000327C1000327470023A2E7008327C101B3
:1009D00083A747000327C100631AF7008327C100DC
:1009E00003A787008327C10123A2E7008327C10053
:1009F00023A807008327C10183A707001387F7FFF8
:100A00008327C10123A0E7008327C10183A7070033
:100A1000138507001301010267800000130101FD27
:100A200023261102232481022326A1002324B100BE
:100A30008327C100232EF1008327C101639607009D
:100A4000737004306F000000EF3010418327C10144
:100A500003A407008327C10103A7C7038327C1019C
:100A600083A707049385070013050700EF80D025AF
:100A7000930705003307F4008327C10123A2E70091
:100A80008327C10123AC07028327C10103A7070005
:100A90008327C10123A4E7008327C10103A4070022
:100AA0008327C10183A7C7031387F7FF8327C101EA
:100AB00083A707049385070013050700EF80D02064
:100AC000930705003307F4008327C10123A6E7003D
:100AD0008327C1011307F0FF23A2E7048327C10185
:100AE0001307F0FF23A4E70483278100639A07021A
:100AF0008327C10183A70701638407048327C101FA
:100B00009387070113850700EF20504C130705005A
:100B1000930710006316F702EFF09FA76F004002E3
:100B20008327C1019387070113850700EFF0DFCA10
:100B30008327C1019387470213850700EFF0DFC9C0
:100B4000EF30903593071000138507008320C10212
:100B5000032481021301010367800000130101FDDA
:100B6000232611022326A1002324B10093070600A7
:100B7000A303F100232C01008327C1006396070023
:100B8000737004306F0000008327810063960700B4
:100B9000232E01006F00C001832581000325C100C1
:100BA000EF8090129307050093871700232EF10022
:100BB0008327C1019387470513850700EF50006E17
:100BC000232AA1008327410163820706832781002E
:100BD000639A0700832741010327410123A0E7000F
:100BE0006F00400183274101138747058327410197
:100BF00023A0E700832741010327C10023AEE702BA
:100C0000832741010327810023A0E70493051000F7
:100C100003254101EFF09FE0832741010347710065
:100C20002388E70483274101232CF10083278101D6
:100C300063960700737004306F0000008327810102
:100C4000138507008320C1021301010367800000A0
:100C5000130101FD2326110293070500A307F100EC
:100C600013054005EF508063232EA1008327C101A7
:100C7000638C07088327C10123A207008327C101D2
:100C800023A007008327C10123A407008327C101F4
:100C900023A607008327C10123AC07028327C101D4
:100CA0001307100023AEE7028327C10123A0070426
:100CB0008327C1011307F0FF23A2E7048327C101A3
:100CC0001307F0FF23A4E7048327C1010347F100C2
:100CD0002388E7048327C101938707011385070051
:100CE000EFF09FAF8327C101938747021385070069
:100CF000EFF09FAE9306000013060000930500007E
:100D00000325C101EF00001E8327C10113850700E1
:100D10008320C1021301010367800000130101FD5C
:100D200023261102232481022326A1008327C10048
:100D3000232CF10083278101639607007370043030
:100D40006F0000008327810103A44700EF3000609B
:100D5000930705006312F4048327810183A7C7006A
:100D60001387F7FF8327810123A6E70083278101EB
:100D700083A7C700639C07009306000013060000CA
:100D80009305000003258101EF00C01593071000B3
:100D9000232EF1006F008000232E01008327C10164
:100DA000138507008320C10203248102130101037C
:100DB00067800000130101FD232611022324810214
:100DC0002326A1002324B1008327C100232CF10096
:100DD0008327810163960700737004306F00000061
:100DE0008327810103A44700EF3040569307050095
:100DF0006312F4028327810183A7C70013871700BA
:100E00008327810123A6E70093071000232EF1001A
:100E10006F00C003930600000326810093050000C5
:100E200003258101EF00C058232EA1000327C10133
:100E300093071000631CF7008327810183A7C70075
:100E4000138717008327810123A6E7008327C101A9
:100E5000138507008320C1020324810213010103CB
:100E600067800000130101FD232611022326A10043
:100E70002324B1008327C1006396070073700430F8
:100E80006F000000032781008327C10063F6E7009D
:100E9000737004306F0000001306200093050000FB
:100EA0000325C100EFF09FCB232EA1008327C101B2
:100EB000638807008327C1010327810023ACE70271
:100EC0008327C10163960700737004306F00000030
:100ED0008327C101138507008320C1021301010389
:100EE00067800000130101FC232E11022326A100BC
:100EF0002324B1002322C1002320D1002326010294
:100F00008327C1002324F10283278102639607000F
:100F1000737004306F00000083278100639807001E
:100F20008327810283A707046396070093071000B5
:100F30006F00800093070000639607007370043011
:100F40006F0000000327010093072000631AF700D9
:100F50008327810203A7C703930710006316F700D6
:100F6000930710006F00800093070000639607004E
:100F7000737004306F000000EF30803F930705006E
:100F800063960700832741006396070093071000CC
:100F90006F008000930700006396070073700430B1
:100FA0006F000000EF30406B8327810203A78703A7
:100FB0008327810283A7C7036368F7000327010023
:100FC000930720006310F7060326010083258100A4
:100FD00003258102EF00101C2322A1028327810236
:100FE00083A747026384070283278102938747020E
:100FF00013850700EF20807D13070500930710007D
:10100000631CF700EFF0CFD86F0000018327410287
:1010100063840700EFF0CFD7EF300068930710002C
:101020006F00400F8327410063980700EF30C066D0
:10103000930700006F00000E8327C102639C070026
:101040009307C10113850700EF20501D930710007F
:101050002326F102EF304064EF10D049EF30C05F3B
:101060008327810203A747049307F0FF6316F70065
:101070008327810223A207048327810203A7870411
:101080009307F0FF6316F7008327810223A4070468
:10109000EF308060130741009307C10193050700FB
:1010A00013850700EF20501C93070500639C07047D
:1010B00003258102EF00504693070500638C070269
:1010C00083278102938707010327410093050700C7
:1010D00013850700EF20004A03258102EF00902CC2
:1010E000EF10904393070500E39E07EAEFF04FCA25
:1010F0006FF05FEB03258102EF00D02AEF10D041A3
:101100006FF05FEA03258102EF00D029EF10D04095
:1011100093070000138507008320C1031301010416
:1011200067800000130101FD232611022326A10080
:101130002324B1002322C1002320D1008327C10032
:10114000232CF1008327810163960700737004301C
:101150006F000000832781006398070083278101C7
:1011600083A7070463960700930710006F008000B1
:101170009307000063960700737004306F0000004F
:101180000327010093072000631AF70083278101DA
:1011900003A7C703930710006316F7009307100017
:1011A0006F0080009307000063960700737004309F
:1011B0006F000000EFF00FD593070500232AF10020
:1011C0008327810103A787038327810183A7C7039F
:1011D0006368F70003270100930720006310F708F6
:1011E000032601008325810003258101EF00807A19
:1011F0008327810103A787049307F0FF6310F70497
:101200008327810183A74702638407048327810121
:101210009387470213850700EF20405B9307050083
:101220006388070283274100638407028327410004
:101230001307100023A0E7006F00800183278101BE
:1012400083A78704138717008327810123A4E7045A
:1012500093071000232EF1006F008000232E010061
:101260008327410113850700EFF00FC88327C101D1
:10127000138507008320C10213010103678000006A
:10128000130101FD232611022326A1002324B1000E
:101290008327C100232CF100832781016396070077
:1012A000737004306F0000008327810183A7070457
:1012B00063860700737004306F000000832781018C
:1012C00083A70700639807008327810183A747004E
:1012D00063960700930710006F00800093070000DB
:1012E00063960700737004306F000000EFF08FC149
:1012F00093070500232AF1008327810103A78703B1
:101300008327810183A7C7036372F70883278101BD
:1013100083A78703138717008327810123ACE70284
:101320008327810103A787049307F0FF6310F70465
:101330008327810183A747026384070483278101F0
:101340009387470213850700EF2040489307050065
:101350006388070283278100638407028327810053
:101360001307100023A0E7006F008001832781018D
:1013700083A78704138717008327810123A4E70429
:1013800093071000232EF1006F008000232E010030
:101390008327410113850700EFF00FB58327C101B3
:1013A000138507008320C102130101036780000039
:1013B000130101FC232E11022326A1002324B100D6
:1013C0002322C1002320D100232601028327C1004C
:1013D0002324F1028327810263960700737004308F
:1013E0006F00000083278100639807008327810234
:1013F00083A7070463960700930710006F0080001F
:101400009307000063960700737004306F000000BC
:10141000EF201076930705006396070083274100AD
:1014200063960700930710006F0080009307000089
:1014300063960700737004306F000000EF30C02126
:101440008327810283A787036382070C8327810296
:1014500083A7C7002322F10283258100032581028F
:10146000EF00806B832701006392070683278102C8
:1014700083A787031387F7FF8327810223ACE70243
:101480008327810283A70700639A0700EF30802B30
:10149000130705008327810223A2E7008327810227
:1014A00083A70701638E07048327810293870701BF
:1014B00013850700EF208031130705009307100004
:1014C0006310F704EFF0CF8C6F0080038327810255
:1014D0000327410223A6E7008327810283A747024F
:1014E00063800702832781029387470213850700E1
:1014F000EF20C02D9307050063840700EFF04F89AC
:10150000EF308019930710006F008011832741008E
:1015100063980700EF304018930700006F004010F9
:101520008327C102639C07009307C101138507004D
:10153000EF20C04E930710002326F102EF30C015B4
:10154000EF10407BEF3040118327810203A747044F
:101550009307F0FF6316F7008327810223A2070495
:101560008327810203A787049307F0FF6316F70020
:101570008327810223A40704EF30001213074100E0
:101580009307C1019305070013850700EF20C04DA5
:1015900093070500639E070603258102EF00406F55
:1015A00093070500638E07048327810283A7070042
:1015B000639E0700EF30400A8327810283A747001C
:1015C00013850700EF20D05FEF30000D83278102E5
:1015D00093874702032741009305070013850700FF
:1015E000EF10507903258102EF00C05BEF10C0724D
:1015F00093070500E39407E4EFE09FF96FF01FE421
:1016000003258102EF00005AEF1000716FF01FE315
:1016100003258102EF000059EF10007093070000CE
:10162000138507008320C1031301010467800000B4
:10163000130101FD232611022326A1002324B1005A
:101640002322C1008327C100232CF10083278101BD
:1016500063960700737004306F00000083278100D9
:10166000639807008327810183A707046396070017
:10167000930710006F008000930700006396070037
:10168000737004306F000000EFF0CF879307050000
:10169000232AF1008327810183A787036388070832
:1016A0008325810003258101EF0000478327810105
:1016B00083A787031387F7FF8327810123ACE70202
:1016C0008327810103A747049307F0FF6310F70402
:1016D0008327810183A7070163840704832781018E
:1016E0009387070113850700EF20400E930705003D
:1016F0006388070283274100638407028327410030
:101700001307100023A0E7006F00800183278101E9
:1017100083A74704138717008327810123A2E704C7
:1017200093071000232EF1006F008000232E01008C
:101730008327410113850700EFE01FFB8327C101C9
:10174000138507008320C102130101036780000095
:10175000130101FD232611022326A1002324B10039
:101760008327C100232CF1008327810163960700A2
:10177000737004306F0000008327810063980700B6
:101780008327810183A7070463960700930710004E
:101790006F008000930700006396070073700430A9
:1017A0006F0000008327810183A707046396070069
:1017B000737004306F000000EFE0DFF49307050062
:1017C000232AF1008327810183A78703638A070205
:1017D0008327810183A7C7002328F1008325810087
:1017E00003258101EF004033832781010327010195
:1017F00023A6E70093071000232EF1006F0080005E
:10180000232E01008327410113850700EFE0DFED60
:101810008327C101138507008320C102130101033F
:1018200067800000130101FD232611022326A10079
:101830008327C10063960700737004306F000000B7
:10184000EF2090618327C10083A78703232EF10037
:10185000EF2090648327C101138507008320C10214
:101860001301010367800000130101FD232611020B
:101870002326A1008327C100232EF1008327C10165
:1018800063960700737004306F000000EF20D05C97
:101890008327C10103A7C7038327C10183A7870348
:1018A000B307F740232CF100EF20105F832781015D
:1018B000138507008320C102130101036780000024
:1018C000130101FE2326A1008327C10063960700B0
:1018D000737004306F0000008327C10083A7870363
:1018E000232EF1008327C101138507001301010294
:1018F00067800000130101FD232611022326A100A9
:101900008327C100232EF1008327C10163960700BE
:10191000737004306F0000000325C101EF004052D6
:101920000325C101EF405037130000008320C1029E
:101930001301010367800000130101FF2326A100AA
:101940008327C10083A7C704138507001301010182
:1019500067800000130101FF2326A1002324B100AA
:101960008327C1000327810023A6E704130000009A
:101970001301010167800000130101FF2326A1006C
:101980008327C10083C707051385070013010101E1
:1019900067800000130101FD232611022326A10008
:1019A0002324B1002322C100232E01008327C1007C
:1019B00083A70704639807028327C10083A7070052
:1019C000639807128327C10083A747001385070088
:1019D000EF20D034232EA1008327C10023A20700CB
:1019E0006F00001183274100639407068327C1001D
:1019F00003A787008327C10083A707041386070076
:101A00008325810013050700EF40D03F8327C100E5
:101A100003A787008327C10083A707043307F700C4
:101A20008327C10023A4E7008327C10003A7870001
:101A30008327C10083A74700636CF70A8327C1008F
:101A400003A707008327C10023A4E7006F00400A13
:101A50008327C10003A7C7008327C10083A707040A
:101A6000138607008325810013050700EF40903996
:101A70008327C10003A7C7008327C10083A70704EA
:101A8000B307F0403307F7008327C10023A6E70020
:101A90008327C10003A7C7008327C10083A70700CE
:101AA0006372F7028327C10003A747008327C100A1
:101AB00083A70704B307F0403307F7008327C1006B
:101AC00023A6E70003274100930720006312F702D3
:101AD0008327C10083A78703638C07008327C10086
:101AE00083A787031387F7FF8327C10023ACE7028F
:101AF0008327C10083A78703138717008327C100AB
:101B000023ACE7028327C101138507008320C102AC
:101B10001301010367800000130101FE232E110051
:101B20002326A1002324B1008327C10083A7070433
:101B3000638207068327C10003A7C7008327C1006C
:101B400083A707043307F7008327C10023A6E70014
:101B50008327C10003A7C7008327C10083A74700CD
:101B6000636AF7008327C10003A707008327C1002A
:101B700023A6E7008327C10003A7C7008327C1006E
:101B800083A7070413860700930507000325810038
:101B9000EF405027130000008320C1011301010210
:101BA00067800000130101FE232E11002326A100EF
:101BB000EF20902A6F0000048327C10083A747020B
:101BC000638207048327C1009387470213850700B8
:101BD000EF10D03F9307050063840700EF10D07823
:101BE0008327C10083A787041387F7FF8327C100DA
:101BF00023A4E7048327C10083A78704E34EF0FAF8
:101C00006F008000130000008327C1001307F0FF5E
:101C100023A4E704EF205028EF2010246F000004D5
:101C20008327C10083A70701638207048327C100BC
:101C30009387070113850700EF10503993070500BC
:101C400063840700EF1050728327C10083A7470405
:101C50001387F7FF8327C10023A2E7048327C1006E
:101C600083A74704E34EF0FA6F00800013000000E2
:101C70008327C1001307F0FF23A2E704EF20D02140
:101C8000130000008320C1011301010267800000DE
:101C9000130101FD232611022326A100EF20D01BF2
:101CA0008327C10083A78703639807009307100069
:101CB000232EF1006F008000232E0100EF20D01DA5
:101CC0008327C101138507008320C102130101038B
:101CD00067800000130101FE2326A1008327C100B5
:101CE00063960700737004306F0000008327C10003
:101CF00083A787036398070093071000232EF10042
:101D00006F008000232E01008327C1011385070087
:101D10001301010267800000130101FD2326110257
:101D20002326A100EF2050138327C10003A78703B8
:101D30008327C10083A7C7036318F7009307100028
:101D4000232EF1006F008000232E0100EF20D0141D
:101D50008327C101138507008320C10213010103FA
:101D600067800000130101FE2326A1008327C10024
:101D700063960700737004306F0000008327C10072
:101D800003A787038327C10083A7C7036318F7004E
:101D900093071000232EF1006F008000232E010016
:101DA0008327C1011385070013010102678000002A
:101DB000130101FE2326A1002324B100232E0100DC
:101DC0006F008006178703001307079F8327C10151
:101DD00093973700B307F70083A7070063900704C2
:101DE000178703001307479D8327C1019397370087
:101DF000B307F7000327810023A0E700178703003C
:101E00001307879B8327C10193973700B307F70018
:101E10000327C10023A2E7006F00C0018327C1018F
:101E200093871700232EF1000327C1019307700049
:101E3000E3FAE7F8130000001301010267800000D5
:101E4000130101FE2326A100232E01006F00C00410
:101E500017870300130747968327C101939737001D
:101E6000B307F70083A747000327C1006310F702F9
:101E700017870300130747948327C10193973700FF
:101E8000B307F70023A007006F00C0018327C1013B
:101E900093871700232EF1000327C10193077000D9
:101EA000E3F8E7FA13000000130101026780000065
:101EB000130101FD232611022326A1002324B100D2
:101EC0002322C1008327C100232EF100EF20C07818
:101ED0008327C10103A747049307F0FF6316F700A8
:101EE0008327C10123A207048327C10103A7870415
:101EF0009307F0FF6316F7008327C10123A40704AB
:101F0000EF2080798327C10183A78703639E0700A1
:101F10008327C1019387470203264100832581005F
:101F200013850700EF10007F0325C101EFF09FC765
:101F3000130000008320C102130101036780000029
:101F4000130101FC232E1102232EA100232CB1002A
:101F50002328D1002326E1002324F10023220101BC
:101F60002320110193070600231BF1008327C101E1
:101F700063960700737004306F0000000327C100F0
:101F80009307400063F6E700737004306F000000B1
:101F9000835761018325410013850700EF10D07E30
:101FA0002324A102832781026386071C83278102E1
:101FB00003A7070383566101B70700409387F7FF24
:101FC000B387F60093972700B307F7002322F102A7
:101FD0008327410293F7C7FF2322F102832741029F
:101FE00093F7370063860700737004306F000000BA
:101FF0008357610113870700832601000326C10070
:102000008325810103258102EF1050410326010140
:102010008325C10103254102EFE0CFF0130705003E
:102020008327810223A0E7008327810063880700BC
:10203000832781000327810223A0E700EF20C061EE
:1020400097E701009387075D83A7070013871700B1
:1020500097E701009387075C23A0E70097E701005B
:102060009387474383A707006398070297E7010018
:10207000938747420327810223A0E70097E70100E7
:102080009387475903A70700930710006312F704CB
:10209000EF10904B6F00C00397E7010093874758FC
:1020A00083A707006396070297E701009387873E9F
:1020B00083A7070083A7C7020327C100636AF7004D
:1020C00097E701009387073D0327810223A0E700DC
:1020D00097E701009387C75583A707001387170069
:1020E00097E701009387C75423A0E70097E7010013
:1020F0009387075403A707008327810223A4E704DB
:102100008327810203A7C70297E70100938707513E
:1021100083A7070063FCE7008327810203A7C702A8
:1021200097E701009387874F23A0E7008327810269
:1021300003A7C7029307070093972700B387E70019
:102140009397270017E701001307873F3387E700BE
:1021500083278102938747009385070013050700B3
:10216000EFE0CFEE930710002326F102EF20C052DC
:102170006F00C0009307F0FF2326F1020327C1027E
:10218000930710006318F70297E701009387474908
:1021900083A707006380070297E701009387872FD3
:1021A00083A7070083A7C7020327C10063F4E700E2
:1021B000EFE00FBE8327C102138507008320C10310
:1021C0001301010467800000130101FD23261102A1
:1021D0002326A100EF2040488327C100639A07000F
:1021E00097E701009387072B83A707006F00800004
:1021F0008327C100232EF1008327C1019387470065
:1022000013850700EFE0CFF88327C10183A787027A
:10221000638A07008327C10193878701138507001D
:10222000EFE00FF78327C1019387470093850700ED
:1022300017E501001305453BEFE04FE197E701008B
:102240009387C73B83A707001387170097E7010011
:102250009387C73A23A0E70097E701009387473D9C
:1022600083A707001387170097E701009387473C70
:1022700023A0E700EF20404297E701009387473A09
:1022800083A707006382070497E7010093878720ED
:1022900083A707000327C1016312F70297E7010034
:1022A0009387873983A7070063860700737004301C
:1022B0006F000000EFE0CFAD6F000001EF20C039EC
:1022C000EF208001EF20403D130000008320C10279
:1022D0001301010367800000130101FD2326110291
:1022E0002326A1002324B100232E01008327C1004F
:1022F00063960700737004306F000000832781002D
:1023000063960700737004306F00000097E70100C8
:102310009387873283A707006386070073700430B2
:102320006F000000EF00101D97E701009387C72E94
:1023300083A70700232CF1008327C10083A7070090
:1023400003278100B307F700232AF1008327C10088
:1023500083A70700032781016376F7028327C10063
:1023600083A70700032741016370F7040327410196
:102370008327810163FAE70293071000232EF100FF
:102380006F0080028327C10083A707000327410154
:102390006368F700032741018327810163F6E700A3
:1023A00093071000232EF1008327C100032741016A
:1023B00023A0E7008327C1016382070297E701009A
:1023C0009387470D83A7070093874700138507006E
:1023D000EFE00FDC03254101EF10502FEF00D01389
:1023E0002328A1008327010163940700EFE04F9A9F
:1023F000130000008320C102130101036780000065
:10240000130101FD232611022326A100232E010022
:102410008327C1006380070697E701009387C721E0
:1024200083A7070063860700737004306F00000005
:10243000EF00500C97E701009387071E83A7070062
:102440000327C100B307F700232CF10097E7010031
:102450009387470483A707009387470013850700E6
:10246000EFE00FD303258101EF105026EF00D00AD3
:10247000232EA1008327C10163940700EFE04F9151
:10248000130000008320C1021301010367800000D4
:10249000130101FD232611022326A1008327C10079
:1024A000232CF100832781016396070073700430A9
:1024B0006F00000097E701009387C7FD83A707001F
:1024C000032781016316F700232E01006F00400AE5
:1024D000EF2080188327810183A74701232AF10079
:1024E000EF20801B97E701009387470E83A7070023
:1024F00003274101630CF70097E701009387470D1D
:1025000083A70700032741016318F7009307200002
:10251000232EF1006F00C0050327410197E701005A
:102520009387070E6314F7028327810183A787022D
:102530006398070093073000232EF1006F004003DB
:1025400093072000232EF1006F0080020327410132
:1025500097E70100938747096318F7009307400046
:10256000232EF1006F00C00093071000232EF1000E
:102570008327C101138507008320C10213010103D2
:1025800067800000130101FD232611022326A1000C
:10259000EF20800C8327C100639A070097E70100B2
:1025A000938747EF83A707006F0080008327C10050
:1025B000232EF1008327C10183A7C702232CF1003A
:1025C000EF20800D83278101138507008320C1023E
:1025D0001301010367800000130101FD232611028E
:1025E0002326A100EFE00F9293070500232EF100B0
:1025F0008327C100639A070097E70100938787E963
:1026000083A707006F0080008327C100232CF100FF
:102610008327810183A7C702232AF1008327C101F1
:1026200013850700EFE04F8C8327410113850700D6
:102630008320C1021301010367800000130101FD23
:10264000232611022326A1002324B100232E0100FA
:10265000032781009307400063F6E700737004309E
:102660006F000000032781009307400063F6E70036
:10267000930740002324F100EF10107E8327C10050
:10268000639A070097E701009387C7E083A70700D5
:102690006F0080008327C100232CF1008327810174
:1026A00083A70705232AF10003274101832781001F
:1026B000630EF716032781008327410163FEE702BB
:1026C00097E70100938707DD83A7070003278101B0
:1026D0006302F70497E701009387C7DB83A707002E
:1026E00083A7C702032781006366F70293071000E0
:1026F000232EF1006F00000297E70100938787D92E
:1027000083A70700032781016316F70093071000D2
:10271000232EF1008327810183A7C7022328F1001C
:102720008327810103A707058327810183A7C702A8
:102730006318F700832781010327810023A6E7029E
:10274000832781010327810023A8E70483278101D0
:1027500083A7870163CC07001307500083278100FC
:102760003307F7408327810123ACE70083278101EA
:1027700083A64701032701019307070093972700CA
:10278000B387E7009397270017E70100130747DB9C
:10279000B387E7006396F600930710006F00800090
:1027A00093070000638C0706832781019387470006
:1027B00013850700EFE0CF9D8327810103A7C702A0
:1027C00097E70100938787E583A7070063FCE7008D
:1027D0008327810103A7C70297E70100938707E4D6
:1027E00023A0E7008327810103A7C70293070700FF
:1027F00093972700B387E7009397270017E7010017
:10280000130707D43387E7008327810193874700A5
:102810009385070013050700EFE04F830327C101ED
:10282000930710006314F700EFD09FD6EF10D06627
:10283000130000008320C102130101036780000020
:10284000130101FD232611022326A100EF10D06001
:102850008327C100639A070097E70100938787C326
:1028600083A707006F0080008327C100232EF1009B
:102870008327C1019387470013850700EFE04F913D
:102880008327C10183A78702638A07008327C101C9
:102890009387870113850700EFE08F8F8327C1019E
:1028A000938747009385070017E50100130545D579
:1028B000EFD0DFF9EF10505E97E70100938787BDF7
:1028C00083A707000327C1016314F70697E70100F8
:1028D000938707D583A707006382070297E7010064
:1028E000938787D583A7070063860700737004303A
:1028F0006F000000EFD0DFC96F00400597E70100CF
:10290000938707D003A7070097E70100938787D035
:1029100083A70700631AF70097E70100938787B73B
:1029200023A007006F008002EF0090286F000002D4
:1029300097E701009387C7CE83A707006388070046
:10294000EF109051EF105019EF10105513000000C8
:102950008320C1021301010367800000130101FEFF
:102960002326A100232E01008327C100232CF10080
:102970008327C10063960700737004306F00000066
:102980008327810103A7470197E70100938747C782
:102990006316F700930710006F0080009307000094
:1029A000638E07028327810103A7870297E701004F
:1029B000938747C26304F7028327810183A78702B5
:1029C00063960700930710006F00800093070000D4
:1029D0006386070093071000232EF1008327C101AF
:1029E000138507001301010267800000130101FD38
:1029F000232611022326A1008327C100232EF100E4
:102A00008327C10063960700737004306F000000D5
:102A10008327C1016384070C97E70100938787A789
:102A200083A707000327C101630AF70AEF10D0420A
:102A30000325C101EFF09FF2130705009307100073
:102A4000631CF7088327C10193874700138507009C
:102A5000EFD01FF48327C10103A7C70297E7010046
:102A60009387C7BB83A7070063FCE7008327C101E7
:102A700003A7C70297E70100938747BA23A0E7009F
:102A80008327C10103A7C702930707009397270075
:102A9000B387E7009397270017E70100130747AABA
:102AA0003387E7008327C101938747009385070099
:102AB00013050700EFD09FD98327C10103A7C702E1
:102AC00097E701009387079D83A7070083A7C702A5
:102AD0006364F700EFD0DFABEF10103C1300000091
:102AE0008320C1021301010367800000130101FD6F
:102AF000232611022326A100232E01008327C100D3
:102B0000232CF1008327C100639607007370043003
:102B10006F000000EFD01FBF93070500232AF100CC
:102B200003258101EFF09FE31307050093071000D1
:102B30006314F70C97E70100938707B083A707009A
:102B40006390070A8327810103A7C70297E7010063
:102B50009387479483A7070083A7C7026366F7009C
:102B600093071000232EF1008327810193874700EC
:102B700013850700EFD0DFE18327810103A7C70298
:102B800097E70100938787A983A7070063FCE70005
:102B90008327810103A7C70297E70100938707A84E
:102BA00023A0E7008327810103A7C702930707003B
:102BB00093972700B387E7009397270017E7010053
:102BC000130707983387E70083278101938747001E
:102BD0009385070013050700EFD05FC76F00C001A2
:102BE00083278101938787019385070017E50100FB
:102BF0001305459EEFD09FC583274101138507002C
:102C0000EFD09FAE8327C101138507008320C10247
:102C10001301010367800000130101FE232E110040
:102C2000930800001308000093070000130700003A
:102C3000930600001306004097D501009385853C5C
:102C400017150000130505FBEFF08FAF2326A10039
:102C50000327C100930710006316F700EF20C03A66
:102C60002326A1000327C10093071000631EF7026B
:102C70007370043097E701009387C79B1307F0FF39
:102C800023A0E70097E701009387879913071000B7
:102C900023A0E70097E701009387079823A0070088
:102CA000EFD04FF46F0040018327C1006396070007
:102CB000737004306F000000130000008320C10116
:102CC0001301010267800000130101FF2326110098
:102CD0007370043097E701009387879423A007005F
:102CE000EFD09F82130000008320C1001301010177
:102CF0006780000097E701009387079483A7070088
:102D00001387170097E701009387079323A0E70035
:102D10001300000067800000130101FE232E110044
:102D20002326010097E701009387079183A70700F7
:102D300063960700737004306F000000EF10D0112D
:102D400097E701009387478F83A707001387F7FF53
:102D500097E701009387478E23A0E70097E70100DC
:102D60009387878D83A707006394071697E7010071
:102D70009387478A83A70700638C07146F00800C32
:102D800097E701009387078583A7C70083A7C7003C
:102D90002324F1008327810093878701138507008F
:102DA000EFD01FBF8327810093874700138507005B
:102DB000EFD01FBE8327810003A7C70297E701005A
:102DC0009387C78583A7070063FCE70083278100FB
:102DD00003A7C70297E701009387478423A0E70072
:102DE0008327810003A7C702930707009397270053
:102DF000B387E7009397270017D70100130747749D
:102E00003387E70083278100938747009385070076
:102E100013050700EFD09FA38327810003A7C702F4
:102E200097D701009387076783A7070083A7C70287
:102E3000636AF70097D701009387077F1307100095
:102E400023A0E70097D701009387C77883A70700DF
:102E5000E39807F297D701009387C77C83A7070001
:102E6000638807046F00C003EF00002B9307050081
:102E7000638A070097D701009387077B1307100029
:102E800023A0E70097D701009387C77983A707009E
:102E90001387F7FF97D701009387C77823A0E70030
:102EA00097D701009387077883A70700E39E07FA67
:102EB00097D701009387477703A707009307100070
:102EC0006318F700930710002326F100EFD04FECB2
:102ED000EF10807C8327C100138507008320C10188
:102EE0001301010267800000130101FE232E11006F
:102EF000EF10807697D701009387077283A70700AA
:102F00002326F100EF1040798327C10013850700C5
:102F10008320C1011301010267800000130101FE3B
:102F2000232E1100EFD00FFE930705002326F1009A
:102F300097D701009387476E83A707002324F100EA
:102F40008327C10013850700EFD00FFA8327810084
:102F5000138507008320C10113010102678000006F
:102F600097D701009387076B83A707001385070096
:102F700067800000130101FD232611022326A10012
:102F80002324B1002322C100232E01009307500007
:102F9000232CF100EFF01FD697D7010093878767A6
:102FA00083A7070003278100636CF714832781013F
:102FB0009387F7FF232CF1008327C10193975700D4
:102FC0000327C100B306F700032781019307070019
:102FD00093972700B387E7009397270017D701003F
:102FE00013070756B387E700130610009385070001
:102FF00013850600EF108004130705008327C10125
:10300000B387E700232EF10083278101E39007FABD
:103010008327C101939757000327C1003307F700A7
:1030200097D701009387875A83A7070013062000CC
:103030009385070013050700EF10400013070500F4
:103040008327C101B387E700232EF1008327C10145
:10305000939757000327C1003307F70097D7010064
:103060009387075783A7070013062000938507005F
:1030700013050700EF00907C130705008327C101AB
:10308000B387E700232EF1008327C10193975700F0
:103090000327C100B307F7001306400097D50100CE
:1030A0009385855413850700EF00507913070500B9
:1030B0008327C101B387E700232EF1008327C101D5
:1030C000939757000327C100B307F700130630009A
:1030D00097D501009385C55213850700EF00107640
:1030E000130705008327C101B387E700232EF100F2
:1030F00083274100638607008327410023A0070040
:10310000EFF09FC18327C101138507008320C1020F
:103110001301010367800000130101FD2326110242
:10312000232E010097D701009387075183A707003B
:10313000639C072297D701009387074E83A7070058
:103140001387170097D701009387074D23A0E70047
:1031500097D701009387474C83A70700232CF100E2
:1031600083278101639C070697D701009387074651
:1031700083A7070083A707006386070073700430E6
:103180006F00000097D701009387474483A707008B
:10319000232AF10097D701009387874303A70700ED
:1031A00097D701009387874223A0E70097D70100B4
:1031B000938707420327410123A0E70097D7010027
:1031C0009387C74683A707001387170097D7010087
:1031D0009387C74523A0E700EF10001097D70100A1
:1031E0009387474583A7070003278101636CF71284
:1031F00097D701009387873D83A7070083A7070020
:1032000063960700930710006F008000930700008B
:10321000638C070097D701009387C7411307F0FF1E
:1032200023A0E7006F00001097D701009387073AAB
:1032300083A7070083A7C70083A7C7002328F1003F
:103240008327010183A747002326F100032781017B
:103250008327C100637CF70097D701009387873DE0
:103260000327C10023A0E7006F00C00B83270101E3
:103270009387470013850700EFD08FF18327010163
:1032800083A78702638A0700832701019387870149
:1032900013850700EFD0CFEF8327010103A7C702F3
:1032A00097D701009387873783A7070063FCE70060
:1032B0008327010103A7C70297D701009387073629
:1032C00023A0E7008327010103A7C7029307070094
:1032D00093972700B387E7009397270017D701003C
:1032E000130707263387E7008327010193874700E9
:1032F0009385070013050700EFD04FD58327010101
:1033000003A7C70297D701009387C71883A70700B1
:1033100083A7C702E36EF7EC93071000232EF1009A
:103320006FF01FED97D701009387C71683A707009B
:1033300003A7C70297D6010093868620930707004C
:1033400093972700B387E70093972700B387F6008A
:1033500003A707009307100063F6E7029307100026
:10336000232EF1006F00000297D701009387872B6F
:1033700083A707001387170097D701009387872A31
:1033800023A0E70097D701009387072A83A70700A8
:103390006386070093071000232EF1008327C101E5
:1033A000138507008320C102130101036780000019
:1033B000130101FE232E110097D701009387C72721
:1033C00083A70700638C070097D701009387C72561
:1033D0001307100023A0E7006F00C01897D7010063
:1033E0009387872423A0070097D701009387870A34
:1033F00083A7070083A707032326F100B7A7A5A586
:103400009387575A2324F1008327C10083A707001D
:10341000032781006310F7048327C10093874700C7
:1034200083A70700032781006316F7028327C100E3
:103430009387870083A7070003278100631CF70099
:103440008327C1009387C70083A707000327810054
:103450006302F70697D701009387C70303A7070006
:1034600097D701009387070383A707009387470334
:103470009385070013050700EF40001F6F008003CE
:1034800097D701009387871983A7070063960700E2
:10349000737004306F00000097D7010093870718FE
:1034A00083A707001387F7FF97D7010093870717B4
:1034B00023A0E70097D701009387471603A70700CB
:1034C00097D601009386C6079307070093972700B6
:1034D000B387E70093972700B387F60083A7070019
:1034E000E38007FA97D701009387471303A70700E4
:1034F0009307070093972700B387E7009397270068
:1035000017D701001307C703B387E7002322F10091
:103510008327410083A7470003A747008327410073
:1035200023A2E7008327410003A747008327410028
:1035300093878700631CF7008327410083A7470018
:1035400003A747008327410023A2E7008327410008
:1035500083A7470003A7C70097D70100938787F386
:1035600023A0E700130000008320C1011301010222
:1035700067800000130101FD232611022326A1000C
:103580002324B1008327C1006396070073700430C1
:103590006F00000097D701009387C7EF83A707004C
:1035A00093878701938507000325C100EFD0CFB132
:1035B00097D70100938707EE83A7070093874700FB
:1035C00013850700EFD0CFBC032781009307F0FFDE
:1035D0006314F70297D701009387C7EB83A707000F
:1035E000938747009385070017D501001305450110
:1035F000EFD0CFA56F00400297D701009387C70196
:1036000083A7070003278100B307F700232EF100EB
:103610000325C101EF00900B130000008320C102BD
:103620001301010367800000130101FD232611022D
:103630002326A1002324B1002322C1008327C10037
:1036400063960700737004306F00000097D7010085
:10365000938787FE83A70700639607007370043083
:103660006F00000097D701009387C7E283A7070088
:10367000832681003707008033E7E60023ACE700AC
:1036800097D70100938707E183A7070093878701F6
:10369000938507000325C100EFD04F9B97D701000A
:1036A000938747DF83A707009387470013850700A9
:1036B000EFD00FAE032741009307F0FF6314F7022A
:1036C00097D70100938707DD83A7070093874700FB
:1036D0009385070017D50100130585F2EFD00F97EA
:1036E0006F00400297D70100938707F383A7070075
:1036F00003274100B307F700232EF1000325C10182
:10370000EF00C07C130000008320C10213010103FD
:1037100067800000130101FD232611022326A1006A
:103720002324B1002322C1008327C1006396070030
:10373000737004306F00000097D70100938787D51E
:1037400083A7070093878701938507000325C1009E
:10375000EFD0CF8F97D701009387C7D383A70700F8
:103760009387470013850700EFD08FA203274100FE
:10377000930710006314F70297D70100938787D14E
:1037800083A70700938747009385070017D501009B
:10379000130505E7EFD08F8B6F00400297D701002C
:1037A000938787E783A7070003278100B307F70004
:1037B000232EF1000325C101EF004071130000002A
:1037C0008320C1021301010367800000130101FD82
:1037D000232611022326A1008327C10083A7C70047
:1037E00083A7C700232CF10083278101639607007C
:1037F000737004306F000000832781019387870175
:1038000013850700EFD0CF9897D701009387C7E2C1
:1038100083A70700639E07068327810193874700DC
:1038200013850700EFD0CF968327810103A7C70236
:1038300097D70100938787DE83A7070063FCE70023
:103840008327810103A7C70297D70100938707DD6C
:1038500023A0E7008327810103A7C702930707007E
:1038600093972700B387E7009397270017D70100A6
:10387000130707CD3387E70083278101938747002C
:103880009385070013050700EFC05FFC6F00C001C0
:1038900083278101938787019385070017D501004E
:1038A000130545D3EFC09FFA8327810103A7C70201
:1038B00097D70100938707BE83A7070083A7C70296
:1038C00063F0E70293071000232EF10097D7010061
:1038D000938787D51307100023A0E7006F008000AF
:1038E000232E01008327C101138507008320C10215
:1038F0001301010367800000130101FD232611025B
:103900002326A1002324B10097D701009387C7D2B3
:1039100083A7070063960700737004306F000000F0
:1039200003278100B70700803367F7008327C100B2
:1039300023A0E7008327C10083A7C700232CF10041
:103940008327810163960700737004306F000000C5
:103950000325C100EFD0CF838327810193874700E0
:1039600013850700EFD0CF828327810103A7C70209
:1039700097D70100938787CA83A7070063FCE700F6
:103980008327810103A7C70297D70100938707C93F
:1039900023A0E7008327810103A7C702930707003D
:1039A00093972700B387E7009397270017D7010065
:1039B000130707B93387E7008327810193874700FF
:1039C0009385070013050700EFC05FE88327810197
:1039D00003A7C70297D701009387C7AB83A7070048
:1039E00083A7C70263F0E70293071000232EF100BC
:1039F00097D70100938747C31307100023A0E70060
:103A00006F008000232E01008327C101138507006A
:103A10008320C1021301010367800000130101FF2D
:103A20002326A1008327C10063960700737004302A
:103A30006F00000097D70100938747BF03A70700D7
:103A40008327C10023A0E70097D701009387C7BC55
:103A500003A707008327C10023A2E700130000008B
:103A60001301010167800000130101FD23261102EB
:103A70002326A1002324B1008327C10063960700F9
:103A8000737004306F000000832781006396070085
:103A9000737004306F000000EF00103C97D70100F6
:103AA000938787B783A70700232CF1008327810022
:103AB00003A707009307F0FF6316F700232E01000A
:103AC0006F0000098327C10003A7070097D70100F3
:103AD0009387C7B583A707006300F7028327C10058
:103AE00083A74700032781016368F700930710004D
:103AF000232EF1006F00C0058327C10083A7470074
:103B0000032781013307F7408327810083A707003C
:103B1000637CF7028327810003A707008327C10086
:103B200083A6470083278101B387F6403307F70058
:103B30008327810023A0E7000325C100EFF01FEEDB
:103B4000232E01006F00C00093071000232EF10008
:103B5000EF0090348327C101138507008320C10241
:103B6000130101036780000097D701009387C7AB5B
:103B70001307100023A0E700130000006780000077
:103B8000130101FE2326A1008327C100638E0700D5
:103B90008327C100232CF1008327810183A7C70459
:103BA000232EF1006F008000232E01008327C10126
:103BB000138507001301010267800000130101FE55
:103BC0002326A1002324B1008327C100638C0700B2
:103BD0008327C100232EF1008327C1010327810021
:103BE00023A6E70413000000130101026780000010
:103BF000130101FE232E11002326A100EF00002156
:103C000097D701009387C79303A707009307100076
:103C1000E3F6E7FEEFC0DF976FF05FFE130101FCF4
:103C2000232E1102232EA100232CB100232AC10030
:103C30002328D100930707002317F1002326010250
:103C40006F004004032781018327C102B307F700F7
:103C500003C707008326C1018327C102B387F6008B
:103C6000238AE702032781018327C102B307F700F4
:103C700083C70700638007028327C1029387170069
:103C80002326F1020327C1029307F000E3FCE7FAC1
:103C90006F008000130000008327C101A381070487
:103CA000032741019307400063F6E70093074000B4
:103CB000232AF1008327C1010327410123A6E7023C
:103CC0008327C1010327410123A8E7048327C101FA
:103CD00023AA07048327C1019387470013850700A0
:103CE000EFC01FB58327C1019387870113850700A4
:103CF000EFC01FB48327C1010327C10123A8E70038
:103D000013075000832741013307F7408327C10180
:103D100023ACE7008327C1010327C10123A2E702E7
:103D20008327C10123A207048327C10123AC070411
:103D30008327C10123AE0704130000008320C103C1
:103D40001301010467800000130101FE232E1100FE
:103D5000232601006F0080030327C100930707009B
:103D600093972700B387E7009397270017C70100B1
:103D70001307077DB387E70013850700EFC0DFA5B2
:103D80008327C100938717002326F1000327C10072
:103D900093074000E3F2E7FC17D501001305858087
:103DA000EFC09FA317D5010013050581EFC0DFA267
:103DB00017D5010013050582EFC01FA217D501001A
:103DC00013058582EFC05FA117D501001305458358
:103DD000EFC09FA097C701009387477F17C70100D7
:103DE0001307477C23A0E70097C701009387477E0E
:103DF00017C701001307477C23A0E700130000004A
:103E00008320C1011301010267800000130101FE3C
:103E1000232E11006F008009EFE0DFED97C701004E
:103E20009387877C83A7070093B7170093F7F70F53
:103E30002326F100EFE05FEE8327C10063980706B9
:103E4000EF00900197C701009387077A83A7C70007
:103E500083A7C7002324F1008327810093874700AD
:103E600013850700EFC0DFB297C701009387877AF9
:103E700083A707001387F7FF97C701009387877908
:103E800023A0E70097C701009387477783A7070020
:103E90001387F7FF97C701009387477623A0E700B2
:103EA000EF00807F03258100EF00C03F97C701002E
:103EB0009387C77483A70700E39007F613000000F9
:103EC0008320C1011301010267800000130101FE7C
:103ED000232E11002326A10097C701009387875B3B
:103EE00083A707000327C10023A2E70097C70100AB
:103EF0009387877283A707000327C1006378F702BF
:103F000097C701009387C76C03A7070097C70100F5
:103F10009387475883A70700938747009385070037
:103F200013050700EFC05F9A6F00000597C70100F7
:103F30009387C76903A7070097C701009387875531
:103F400083A70700938747009385070013050700A1
:103F5000EFC09F9797C701009387C76D83A707009E
:103F60000327C100637AF70097C701009387876C26
:103F70000327C10023A0E700130000008320C10134
:103F80001301010267800000130101FD23261102C5
:103F9000930705002324B1002317F1008327810034
:103FA000639E07008357E10093972700138507005E
:103FB000EF20C02E930705006F008000832781004B
:103FC000232CF10083278101638A07021305000671
:103FD000EF20C02C232EA1008327C101638A070094
:103FE0008327C1010327810123A8E7026F00400155
:103FF00003258101EF20404A6F008000232E01003D
:104000008327C101638207028327C10103A7070336
:104010008357E10093972700138607009305500A02
:1040200013050700EF20006A8327C10113850700ED
:104030008320C1021301010367800000130101FC0A
:10404000232E1102232C81022326A1002324B10058
:104050002322C100232601028327810083A70700B2
:104060006388071C832781002324F10283278102B0
:1040700083A7470003A747008327810223A2E70005
:104080008327810203A74700832781029387870044
:10409000631CF7008327810283A7470003A747001B
:1040A0008327810223A2E7008327810283A7470099
:1040B00083A7C7002322F102832781002320F10276
:1040C0008327010283A7470003A747008327010234
:1040D00023A2E7008327010203A7470083270102E9
:1040E00093878700631CF7008327010283A747009B
:1040F00003A747008327010223A2E70083270102C9
:1041000083A7470083A7C700232EF1008327C1029E
:10411000939757000327C100B307F7000327C10196
:1041200023A0E7008327C102939757000327C1000C
:10413000B307F7000327C1011307470323A2E700D2
:104140008327C102939757000327C100B307F700E5
:104150000327C1010327870423A4E7008327C102A3
:10416000939757000327C100B307F70003274100C7
:1041700023A6E7008327C102939757000327C100B6
:10418000B307F7000327C1010327C70223A8E700ED
:1041900003274100930730006314F7028327C1010E
:1041A00083A78702638E07008327C1029397570076
:1041B0000327C100B307F7001307200023A6E70079
:1041C0008327C102939757000327C100B307F70065
:1041D0000327C1010327070523AAE7008327C1029C
:1041E000939757000327C100B307F70023AC0700DC
:1041F0008327C10183A607038327C1029397570032
:104200000327C1003304F70013850600EF00C00345
:1042100093070500231EF4008327C102938717002C
:104220002326F1020327C10183274102E316F7E8A1
:104230008327C102138507008320C1030324810360
:104240001301010467800000130101FE2326A10071
:10425000232E01006F00C0018327C1009387170040
:104260002326F1008327C10193871700232EF10035
:104270008327C10003C707009307500AE30EF7FC2A
:104280008327C10193D72700232EF1008327C10183
:104290009397070193D707011385070013010102C4
:1042A00067800000130101FE232E11002326A100C8
:1042B0008327C10083A7070313850700EF20C01DD4
:1042C0000325C100EF20401D130000008320C10121
:1042D0001301010267800000130101FF97C701006D
:1042E0009387C72E83A7070083A70700639607005D
:1042F000930710006F00800093070000638C070095
:1043000097C70100938707331307F0FF23A0E70047
:104310006F00000397C701009387472B83A707000F
:1043200083A7C70083A7C7002326F1008327C10006
:1043300003A7470097C701009387C72F23A0E70073
:10434000130000001301010167800000130101FF49
:1043500097C701009387071483A707002326F1005E
:104360008327C10013850700130101016780000046
:10437000130101FF97C701009387872A83A70700CE
:1043800063980700930710002326F1006F00400296
:1043900097C701009387472A83A707006398070000
:1043A000930720002326F1006F00800023260100E0
:1043B0008327C100138507001301010167800000F6
:1043C000130101FD232611022326A1008327C1002A
:1043D000232EF1008327C100638A07128327C101BE
:1043E00003A7C70297C701009387C70A83A70700DF
:1043F00083A7C702637CF7108327C10183A78701C6
:1044000063C2070297C701009387C70883A7070005
:1044100083A7C702130750003307F7408327C10162
:1044200023ACE7008327C10183A647018327C1018D
:1044300003A7C7029307070093972700B387E700F6
:104440009397270017C701001307870FB387E7006B
:104450006396F600930710006F008000930700003A
:10446000638A07088327C1019387470013850700E4
:10447000EFC00FD297C701009387C70183A707003A
:1044800003A7C7028327C10123A6E7028327C1012F
:1044900003A7C70297C701009387471883A70700A0
:1044A00063FCE7008327C10103A7C70297C7010088
:1044B0009387C71623A0E7008327C10103A7C7027C
:1044C0009307070093972700B387E7009397270088
:1044D00017C701001307C7063387E7008327C10109
:1044E000938747009385070013050700EFC00FB6B9
:1044F0006F00C00197C701009387C7F983A7070022
:1045000003A7C7028327C10123A6E7021300000007
:104510008320C1021301010367800000130101FD24
:10452000232611022326A1008327C100232CF1009A
:10453000232E01008327C1006386071097C701005F
:10454000938747F583A70700032781016306F700D8
:10455000737004306F0000008327810183A7470533
:1045600063960700737004306F0000008327810199
:1045700083A747051387F7FF8327810123AAE70451
:104580008327810103A7C7028327810183A707052A
:10459000630AF70A8327810183A747056394070A03
:1045A000832781019387470013850700EFC04FBE23
:1045B0008327810103A707058327810123A6E7023B
:1045C0008327810183A7C702130750003307F740F1
:1045D0008327810123ACE7008327810103A7C7025A
:1045E00097C701009387870383A7070063FCE70051
:1045F0008327810103A7C70297C70100938707029A
:1046000023A0E7008327810103A7C70293070700C0
:1046100093972700B387E7009397270017C70100F8
:10462000130707F23387E700832781019387470049
:104630009385070013050700EFC04FA193071000F3
:10464000232EF1008327C101138507008320C102B7
:1046500013010103678000007370043097C70100E5
:10466000938707FC83A707006384070297C70100AD
:10467000938747E283A7070003A7470413071700A0
:1046800023A2E70497C701009387C7E083A7070029
:10469000130000006780000097C70100938747F868
:1046A00083A707006384070497C70100938787DE09
:1046B00083A7070083A74704638A070297C70100FF
:1046C000938747DD83A7070003A747041307F7FF76
:1046D00023A2E70497C701009387C7DB83A70700DE
:1046E00083A747046394070073600430130000003D
:1046F00067800000130101FF97C70100938787D9E6
:1047000083A7070083A787012326F10097C701002D
:10471000938747D883A7070003A7C70297C701005D
:10472000938747D783A70700930650003387E64057
:1047300023ACE7008327C1001385070013010101A3
:104740006780000097C701009387C7D483A707003D
:10475000638E070097C701009387C7D383A707001D
:1047600003A747051307170023AAE70497C701000B
:10477000938747D283A7070013850700678000004F
:10478000130101FD232611022326A1002324B100D9
:10479000EFF09FEC97C701009387C7CF83A707006F
:1047A00083A787056396070897C70100938787CE7D
:1047B00083A707001307100023AEE70483278100B7
:1047C0006388070697C701009387C7CC83A70700B4
:1047D0009387470013850700EFC08F9B0327810055
:1047E0009307F0FF6314F70297C70100938787CA06
:1047F00083A70700938747009385070017C501002B
:10480000130505E0EFC08F846F00400297C70100D9
:10481000938787E083A7070003278100B307F7008A
:10482000232EF1000325C101EFF04FEAEFB05FD670
:10483000EFF09FE6EFF05FE297C70100938787C52F
:1048400083A7070083A78705232CF1008327810115
:10485000638C07028327C100638C070097C70100A0
:10486000938747C383A7070023AC07046F00C001E9
:1048700097C70100938707C283A7070003A787058F
:104880001307F7FF23ACE70497C70100938787C09E
:1048900083A7070023AE0704EFF01FE08327810101
:1048A000138507008320C102130101036780000004
:1048B000130101FD232611022326A1002324B100A8
:1048C0002322C1002320D100EFF01FD997C7010098
:1048D000938747BC83A7070003A7C705930720005A
:1048E0006306F70A97C701009387C7BA83A7070033
:1048F00083A687050327C1001347F7FF33F7E600B8
:1049000023ACE70497C701009387C7B883A70700C4
:104910001307100023AEE70483270100638807060E
:1049200097C70100938707B783A7070093874700BE
:1049300013850700EFC0CF85032701009307F0FF21
:104940006314F70297C701009387C7B483A70700D2
:10495000938747009385070017C50100130545CAD3
:10496000EFB0DFEE6F00400297C701009387C7CA20
:1049700083A7070003270100B307F700232CF100EA
:1049800003258101EFF08FD4EFB09FC0EFF0DFD0AF
:10499000EFF09FCC83274100638E070097C701008B
:1049A000938747AF83A7070003A7870583274100A5
:1049B00023A0E70097C701009387C7AD83A707002F
:1049C00003A7C705930710006316F700232E010005
:1049D0006F00C00297C701009387C7AB83A707008A
:1049E00083A68705032781001347F7FF33F7E60007
:1049F00023ACE70493071000232EF10097C70100B2
:104A0000938747A983A7070023AE0704EFF0DFC809
:104A10008327C101138507008320C102130101030D
:104A200067800000130101FD232611022326A10047
:104A30002324B1002322C1002320D10093071000BA
:104A4000232EF1008327C1006396070073700430A2
:104A50006F0000008327C100232CF100EFF0DFBFBF
:104A600083270100638A07008327810103A7870545
:104A70008327010023A0E7008327810183A7C705BF
:104A8000232AF100832781011307200023AEE704C6
:104A9000032741009307400063ECE70883274100A8
:104AA0001397270097B7010093874756B307F7007E
:104AB00003A7070097B7010093874755B307F7008F
:104AC000678007008327810103A78705832781006B
:104AD0003367F7008327810123ACE7046F004005AB
:104AE0008327810183A78705138717008327810107
:104AF00023ACE7046F00C0038327810103278100F3
:104B000023ACE7046F00C002032741019307200094
:104B1000630AF700832781010327810023ACE704A0
:104B20006F000001232E01006F00800013000000C1
:104B300003274101930710006316F70A83278101B9
:104B40009387470013850700EFB09FE48327810117
:104B500003A7C70297C70100938747AC83A7070045
:104B600063FCE7008327810103A7C70297C7010001
:104B70009387C7AA23A0E7008327810103A7C70261
:104B80009307070093972700B387E70093972700C1
:104B900017C701001307C79A3387E70083278101EE
:104BA000938747009385070013050700EFB01FCADE
:104BB0008327810183A7870263860700737004300F
:104BC0006F0000008327810103A7C70297C7010078
:104BD0009387478C83A7070083A7C70263F4E70086
:104BE000EFB01F9BEFF05FAB8327C1011385070078
:104BF0008320C1021301010367800000130101FC3F
:104C0000232E1102232EA100232CB100232AC10040
:104C10002328D1002326E100930710002326F10268
:104C20008327C10163960700737004306F00000092
:104C30008327C1012324F102EFB0DFAC9307050005
:104C40002322F10283270101638A0700832781025F
:104C500003A787058327010123A0E700832781029B
:104C600083A7C7052320F1028327810213072000B1
:104C700023AEE704032741019307400063ECE708F4
:104C8000832741011397270097B70100938747397E
:104C9000B307F70003A7070097B7010093874738CA
:104CA000B307F700678007008327810203A7870502
:104CB000832781013367F7008327810223ACE70450
:104CC0006F0040058327810283A78705138717009C
:104CD0008327810223ACE7046F00C003832781028E
:104CE0000327810123ACE7046F00C0020327010200
:104CF00093072000630AF7008327810203278101BD
:104D000023ACE7046F000001232601026F0080003E
:104D10001300000003270102930710006314F70E2D
:104D20008327810283A7870263860700737004309C
:104D30006F00000097C701009387079083A70700C3
:104D4000639E070683278102938747001385070028
:104D5000EFB01FC48327810203A7C70297C70100D2
:104D60009387C78B83A7070063FCE7008327810233
:104D700003A7C70297C701009387478A23A0E700CC
:104D80008327810203A7C702930707009397270091
:104D9000B387E7009397270017B701001307477AF7
:104DA0003387E700832781029387470093850700B5
:104DB00013050700EFB09FA96F00C0018327810290
:104DC000938787019385070017C501001305858028
:104DD000EFB0DFA78327810203A7C70297B70100BF
:104DE0009387476B83A7070083A7C70263FCE7008D
:104DF0008327C100638807008327C10013071000C1
:104E000023A0E7008327410213850700EFB0DF8D61
:104E10008327C102138507008320C1031301010406
:104E200067800000130101FD232611022326A10043
:104E30002324B1008327C1006396070073700430F8
:104E40006F0000008327C100232EF100EFB09F8B7D
:104E500093070500232CF1008327C10183A7C70511
:104E6000232AF1008327C1011307200023AEE704A2
:104E70008327C10183A78705138717008327C101F3
:104E800023ACE70403274101930710006314F70ED6
:104E90008327C10183A787026386070073700430EC
:104EA0006F00000097B701009387077983A7070079
:104EB000639E07068327C101938747001385070078
:104EC000EFB01FAD8327C10103A7C70297B7010049
:104ED0009387C77483A7070063FCE7008327C1019A
:104EE00003A7C70297B701009387477323A0E70082
:104EF0008327C10103A7C7029307070093972700E1
:104F0000B387E7009397270017B70100130747639C
:104F10003387E7008327C101938747009385070004
:104F200013050700EFB09F926F00C0018327C101F6
:104F3000938787019385070017B5010013058569DD
:104F4000EFB0DF908327C10103A7C70297B7010025
:104F50009387475483A7070083A7C70263FCE70032
:104F600083278100638807008327810013071000CF
:104F700023A0E7008327810113850700EFB0CFF658
:104F8000130000008320C1021301010367800000A9
:104F9000130101FD232611022326A1008327C1004E
:104FA000232CF10083278101639A070097B7010042
:104FB0009387474E83A707006F00800083278101F6
:104FC000232CF100EFF04FE98327810103A7C705E8
:104FD00093072000631CF7008327810123AE070499
:104FE00093071000232EF1006F008000232E010094
:104FF000EFF08FEA8327C101138507008320C102E8
:105000001301010367800000130101FE232E11002C
:1050100023260100EF00500B97B701009387076527
:1050200083A70700638A07029308000013080000A3
:1050300093070000130720009306000013060040AA
:1050400097B50100938505FF170500001305852E10
:10505000EFC01FEF2326A1008327C100639607003E
:10506000737004306F0000008327C10013850700B0
:105070008320C1011301010267800000130101FCBC
:10508000232E1102232EA100232CB100232AC100BC
:105090002328D1002326E10083278101639607009E
:1050A000232601026F0080061305C002EF10001FC7
:1050B0002326A1028327C102638A0704EF00D000E0
:1050C0008327C1020327C10123A0E7008327C10270
:1050D0000327810123ACE7008327C1020327410195
:1050E00023AEE7008327C1020327010123A0E702C3
:1050F0008327C1020327C10023A2E7028327C1023D
:105100009387470013850700EFB08FF28327810153
:1051100063960700737004306F0000008327C1029C
:10512000138507008320C103130101046780000079
:10513000130101FC232E1102232EA100232CB10008
:10514000232AC1002328D1002326E10023260102BF
:105150008327C10163960700737004306F0000005D
:1051600097B701009387875083A70700638C070ACE
:10517000832781012320F102832741012322F102A9
:105180008327C1012324F1020327810193075000E3
:1051900063C6E706EFF0CF9D1307050093072000D5
:1051A0006318F70297B701009387474C83A707005E
:1051B00013070102930600000326C10093050700B0
:1051C00013850700EFB01FD22326A1026F008005D0
:1051D00097B701009387874983A707001307010248
:1051E00093060000130600009305070013850700CF
:1051F000EFB05FCF2326A1026F00C00297B7010076
:105200009387C74683A70700130701029306000090
:10521000032601019305070013850700EFB09FF0F7
:105220002326A1028327C102138507008320C1031F
:105230001301010467800000130101FE2326A10071
:105240008327C100232EF1008327C1006396070046
:10525000737004306F0000008327C10183A707002B
:10526000138507001301010267800000130101FD8F
:10527000232611022326A1002324B10097B70100A1
:105280009387473E83A7070083A7C70083A7C7006C
:10529000232EF1008327C101938747001385070060
:1052A000EFB00FEF8327C10103A7C70193071000D9
:1052B0006310F7068327C10103A787018327C10075
:1052C000B307F7008326C1000326810093850700FA
:1052D0000325C101EF00802213070500930710008A
:1052E0006318F70213070000930600000326C100AD
:1052F000930500000325C101EFF09FE3232CA100DB
:105300008327810163960700737004306F000000EB
:105310008327C10183A747020325C101E780070056
:10532000130000008320C102130101036780000005
:10533000130101FD232611022326A10093078101F9
:1053400013850700EF00800E232EA1008327810123
:10535000938507000325C101EF00C000EF0000287E
:105360006FF0DFFD130101FD232611022326A100AA
:105370002324B100EFD01F98930781011385070004
:10538000EF004011232EA1008327810163960708B7
:1053900083278100639207020327C1008327C1018D
:1053A00063ECE700EFD05F978325C1010325C100BF
:1053B000EFF0DFEB6F008006832781006380070238
:1053C00097B701009387472A83A7070083A70700A1
:1053D00093B7170093F7F70F2324F10097B7010055
:1053E0009387C72883A607000327C1008327C1012D
:1053F000B307F74003268100938507001385060055
:10540000EFC01FABEFD05F919307050063980700D3
:10541000EFB00F986F008000EFD01F9013000000D6
:105420008320C1021301010367800000130101FE04
:105430002326A10097B701009387C72283A70700FF
:1054400083A7070093B7170093F7F70F1387070099
:105450008327C10023A0E7008327C10083A707009B
:105460006390070297B701009387C71F83A70700C0
:1054700083A7C70083A70700232EF1006F008000D9
:10548000232E01008327C1011385070013010102A8
:1054900067800000130101FD232611022326A100CD
:1054A000EFD09FA4232EA10097B701009387471C3C
:1054B00083A707000327C101637CF700EF00C02B1F
:1054C0008327C1001307100023A0E7006F00C0006E
:1054D0008327C10023A0070097B7010093874719CE
:1054E0000327C10123A0E7008327C101138507001B
:1054F0008320C1021301010367800000130101FD35
:10550000232611022326A1002324B1002322C10057
:105510002320D100232E01008327C100032781000F
:1055200023A2E7008327C1000327C10023A8E700C7
:10553000032781008327410063E6E7040327410036
:10554000832701003307F7408327C10083A7870122
:105550006368F70093071000232EF1006F00C00668
:1055600097B701009387471003A707008327C1005F
:10557000938747009385070013050700EFB0CFB46A
:105580006F0080040327410083270100637EF7003A
:1055900003278100832701006368F7009307100049
:1055A000232EF1006F00400297B701009387870B0D
:1055B00003A707008327C10093874700938507004F
:1055C00013050700EFB04FB08327C1011385070013
:1055D0008320C1021301010367800000130101FD54
:1055E000232611026F0080158327810063C60714EC
:1055F00083270101232EF1008327C10183A74701DF
:10560000638A07008327C10193874700138507003A
:10561000EFB00FB89307410013850700EFF09FE745
:10562000232CA10083278100130790006368F710E3
:105630001397270097B70100938747A0B307F70098
:1056400003A7070097B701009387479FB307F700A9
:10565000678007000327C1008327C10183A7870153
:10566000B307F7000327C100930607000326810153
:10567000938507000325C101EFF05FE813070500DC
:1056800093071000631CF70A8327C10183A7470211
:105690000325C101E78007008327C10103A7C701D4
:1056A00093071000631CF7080327C1008327C1017B
:1056B00083A78701B307F7001307000093060000D4
:1056C00013860700930500000325C101EFF05FA6D4
:1056D000232AA100832741016392070673700430D7
:1056E0006F0000000327C1008327C10123ACE7003E
:1056F0008327C10183A78701639607007370043075
:105700006F0000008327C10103A787018327810160
:10571000B307F700832681010326810193850700E3
:105720000325C101EFF09FDD6F0040010325C1019A
:10573000EF0090566F0080001300000097B7010043
:105740009387C7F283A70700130781009306000021
:10575000130600009305070013850700EFB05FC52F
:1057600093070500E39207E8130000008320C102BD
:105770001301010367800000130101FD23261102BC
:105780006F00C00E97B701009387C7ED83A707008E
:1057900083A7C70083A70700232CF10097B7010058
:1057A000938747EC83A7070083A7C70083A7C70099
:1057B000232AF100832741019387470013850700BF
:1057C000EFB00F9D8327410183A7470203254101C5
:1057D000E78007008327410103A7C7019307100053
:1057E0006316F7088327410183A7870103278101F7
:1057F000B307F7002328F100032701018327810164
:1058000063F0E704832741010327010123A2E70096
:10581000832741010327410123A8E70097B701002F
:10582000938747E403A70700832741019387470035
:105830009385070013050700EFB00F896F00000381
:105840001307000093060000032681019305000062
:1058500003254101EFF0DF8D2326A1008327C1003E
:1058600063960700737004306F00000097B7010063
:10587000938747DF83A7070083A70700E39407F018
:1058800097B70100938707DE83A70700232EF10057
:1058900097B70100938747DD03A7070097B701007B
:1058A000938747DC23A0E70097B701009387C7DB06
:1058B0000327C10123A0E700130000008320C102D9
:1058C0001301010367800000130101FF232611006B
:1058D000EFE09FD897B70100938747D983A70700C8
:1058E0006394070A17B50100130545D5EFA0DFEE55
:1058F00017B501001305C5D5EFA01FEE97B701003E
:10590000938747D617B70100130747D323A0E700B3
:1059100097B70100938747D517B70100130747D3FF
:1059200023A0E700130600009305C0001305400004
:10593000EFB0CFA21307050097B70100938707D3F5
:1059400023A0E70097B70100938747D283A70700FA
:1059500063960700737004306F00000097B7010072
:105960009387C7D083A707006380070297B701001A
:105970009387C7CF83A7070097A501009385856EFE
:1059800013850700EFC0CFC2EFE01FD11300000066
:105990008320C1001301010167800000130101FD94
:1059A000232611022326A1008327C100232EF10004
:1059B0008327C10063960700737004306F000000F6
:1059C000EFE09FC98327C10183A74701B337F000E8
:1059D00093F7F70F232CF100EFE01FCC8327810111
:1059E000138507008320C1021301010367800000B3
:1059F000130101FD232611022326A1008327C100E4
:105A0000232EF1008327C1006396070073700430D2
:105A10006F000000EFE05FC48327C10183A7070286
:105A2000232CF100EFE05FC7832781011385070076
:105A30008320C1021301010367800000130101FDEF
:105A4000232611022326A1002324B1008327C100AD
:105A5000232EF1008327C100639607007370043082
:105A60006F000000EFE05FBF8327C10103278100C3
:105A700023A0E702EFE05FC2130000008320C10211
:105A80001301010367800000130101FE232E1100A2
:105A90001305C001EF0090002326A1008327C10059
:105AA000638E07008327C10023A007008327C1005E
:105AB0009387470013850700EFA01FD28327C100FB
:105AC000138507008320C1011301010267800000D4
:105AD000130101FC232E11022326A1002324B1006F
:105AE0002322C1002320D1008327C1002324F102F7
:105AF0002322010203274100B70700FFB377F70015
:105B000063860700737004306F0000008327410034
:105B100063960700737004306F000000EFE05F854C
:105B2000930705006396070083270100639607002B
:105B3000930710006F008000930700006396070032
:105B4000737004306F000000EFD0CF9A832781027A
:105B500083A707002320F102832581000325C100CC
:105B6000EF00804103270102832781003367F7009C
:105B700083274100B377F70003274100631CF70236
:105B80000327010283278100B367F7002326F10270
:105B90008327810203A707008327410093C7F7FFEC
:105BA0003377F7008327810223A0E7002320010039
:105BB0006F00400483270100638807028327810266
:105BC0009386470003274100B7070005B367F70036
:105BD000032601009385070013850600EFD0DFA49C
:105BE000232601026F0000018327810283A707009B
:105BF0002326F102EFD04F92232EA100832701002C
:105C0000638407088327C10163940700EFA05F98AE
:105C1000EFE05FAE2326A1020327C102B70700020F
:105C2000B377F70063980704EFE01FA3832781028F
:105C300083A707002326F1020327C102832741001F
:105C4000B377F700032741006310F702832781022F
:105C500003A707008327410093C7F7FF3377F700B7
:105C60008327810223A0E700EFE01FA39307100022
:105C70002322F1020327C102B70700019387F7FF30
:105C8000B377F7002326F1028327C10213850700AB
:105C90008320C1031301010467800000130101FB8D
:105CA00023261104232EA100232CB100232AC10096
:105CB0002328D1002326E1008327C101232AF102F2
:105CC000232C0102232801028327C10163960700C8
:105CD000737004306F00000003278101B70700FFD5
:105CE000B377F70063860700737004306F0000001D
:105CF0008327810163960700737004306F000000F2
:105D0000EFE00FE793070500639607008327C100C4
:105D100063960700930710006F0080009307000050
:105D200063960700737004306F000000EFC09FFCA3
:105D30008327410383A707002326F10203260101DD
:105D4000832581010325C102EF00404B2324A102DA
:105D500083278102638C07028327C102232EF1026D
:105D60002326010083274101638807088327410315
:105D700003A707008327810193C7F7FF3377F70055
:105D80008327410323A0E7006F0000078327C1009A
:105D9000639807008327C102232EF1026F00C0051C
:105DA00083274101638A070003278103B7070001A6
:105DB000B367F700232CF10283270101638A0700F0
:105DC00003278103B7070004B367F700232CF10210
:105DD000832741039386470003278101832781039B
:105DE000B367F7000326C1009385070013850600FB
:105DF000EFD09F83232E0102EFC01FF22322A102C6
:105E00008327C10063880708832741026394070042
:105E1000EFA00FF8EFE01F8E232EA1020327C1038E
:105E2000B7070002B377F700639C0704EFE0DF8257
:105E30008327410383A70700232EF10203260101D4
:105E4000832581010325C103EF00403B9307050033
:105E5000638407028327410163800702832741038C
:105E600003A707008327810193C7F7FF3377F70064
:105E70008327410323A0E700EFE01F8223280102CC
:105E80000327C103B70700019387F7FFB377F70034
:105E9000232EF1028327C103138507008320C10449
:105EA0001301010567800000130101FD2326110283
:105EB0002326A1002324B1008327C100232EF10053
:105EC0008327C10063960700737004306F000000E1
:105ED00003278100B70700FFB377F7006386070049
:105EE000737004306F000000EFE00FF78327C101EB
:105EF00083A70700232CF1008327C10103A7070014
:105F00008327810093C7F7FF3377F7008327C10109
:105F100023A0E700EFE04FF88327810113850700F6
:105F20008320C1021301010367800000130101FDFA
:105F3000232611022326A1008327C100232EF1006E
:105F4000EFA04FFC93070500232CF1008327C1012C
:105F500083A70700232AF100832781011385070007
:105F6000EFA08FF883274101138507008320C1022A
:105F70001301010367800000130101FB23261104B4
:105F80002326A1002324B100232C01028327C10072
:105F90002328F102232A01028327C1006396070008
:105FA000737004306F00000003278100B70700FF03
:105FB000B377F70063860700737004306F0000004A
:105FC00083270103938747002326F1028327C10219
:105FD000938787002324F102EFC0DFD18327C1021A
:105FE00083A7C700232EF1028327010303A707001D
:105FF000832781003367F7008327010323A0E7008D
:106000006F00000E8327C10383A747002322F102FC
:106010008327C10383A707002320F102232A01025B
:1060200003270102B70700FFB377F700232EF10023
:1060300003270102B70700019387F7FFB377F70043
:106040002320F1020327C101B7070004B377F7004B
:10605000639207028327010303A707008327010236
:10606000B377F7006388070293071000232AF10231
:106070006F0040028327010303A707008327010263
:10608000B377F700032701026316F70093071000A8
:10609000232AF10283274103638007040327C101F8
:1060A000B7070001B377F700638A0700032781036E
:1060B00083270102B367F700232CF1028327010332
:1060C00003A70700B7070002B367F700938507002F
:1060D0000325C103EFD05F8283274102232EF10203
:1060E0000327C10383278102E31EF7F083270103FF
:1060F00003A707008327810393C7F7FF3377F700D0
:106100008327010323A0E700EFC01FC183270103FA
:1061100083A70700138507008320C104130101052D
:1061200067800000130101FD232611022326A10030
:106130008327C100232EF1008327C10193874700E5
:10614000232CF100EFC01FBB6F00400383278101A8
:1061500003A7C70083278101938787006316F70091
:10616000737004306F0000008327810183A7C7008C
:10617000B705000213850700EFD00FF883278101D0
:1061800083A70700E39407FC0325C101EF00C0309B
:10619000EFC09FB8130000008320C1021301010368
:1061A00067800000130101FE232E11002326A100A9
:1061B0002324B100832581000325C100EFF0DFDB3C
:1061C000130000008320C101130101026780000059
:1061D000130101FE232E11002326A1002324B10068
:1061E000832581000325C100EFF01FCC13000000C0
:1061F0008320C1011301010267800000130101FE29
:106200002326A1002324B1002322C100232E010054
:1062100083274100639007020327C1008327810081
:10622000B377F7006386070293071000232EF1006F
:106230006F0000020327C10083278100B377F700B6
:10624000032781006316F70093071000232EF10047
:106250008327C10113850700130101026780000035
:10626000130101FE2326A1008327C100232CF10086
:106270008327C10063960700232E01006F000001F1
:106280008327810183A78701232EF1008327C10182
:10629000138507001301010267800000130101FC50
:1062A000232E11022326A10023220102EFC09FA466
:1062B000973703009387073D83A70700639C070078
:1062C000EF00002C973703009387C73B130710009C
:1062D00023A0E7008327C100638A07029307800099
:1062E000138707008327C100B387E7002326F10047
:1062F0008327C10093F73700638A07008327C10013
:1063000093F7C7FF938747002326F1008327C10037
:10631000638207160327C100B79701009387B7FF71
:1063200063EAE714973703009387C7342324F10205
:10633000973703009387073483A707002326F102CA
:106340006F0080018327C1022324F1028327C10249
:1063500083A707002326F1028327C10283A74700F2
:106360000327C10063F8E7008327C10283A7070062
:10637000E39A07FC0327C10297370300938707308E
:10638000630AF70E8327810283A7070013078000A3
:10639000B387E7002322F1028327C10203A7070086
:1063A0008327810223A0E7008327C10203A74700B8
:1063B0008327C100B307F7401307800013171700A6
:1063C0006378F7080327C1028327C100B307F700EA
:1063D000232EF1008327C10203A747008327C100B2
:1063E0003307F7408327C10123A2E7008327C102B7
:1063F0000327C10023A2E7008327C10183A7470029
:10640000232CF100973703009387C7262320F1023E
:106410006F0000018327010283A707002320F102F8
:106420008327010283A7070083A747000327810171
:10643000E3E2E7FE8327010203A707008327C101E8
:1064400023A0E700832701020327C10123A0E7005F
:1064500097A701009387470503A707008327C10279
:1064600083A747003307F74097A701009387C70327
:1064700023A0E700EFC05F8A8327410263940700EF
:10648000EF10801D83274102138507008320C1037D
:106490001301010467800000130101FD232611028E
:1064A0002326A1008327C100232CF1008327C100EC
:1064B0006382070A93078000B307F0400327810136
:1064C000B307F700232CF10083278101232AF10071
:1064D000EFC05F828327410183A747002328F10093
:1064E0009737030093870719232EF1006F000001EF
:1064F0008327C10183A70700232EF1008327C10151
:1065000083A7070083A7470003270101E3E2E7FE13
:106510008327C10103A707008327410123A0E700C8
:106520008327C1010327410123A0E70083274101FD
:1065300003A7470097A70100938707F783A70700E2
:106540003307F70097A70100938707F623A0E7001A
:10655000EFC08FFC130000008320C1021301010370
:106560006780000097A70100938707F483A70700BF
:10657000138507006780000013000000678000009B
:10658000130101FF97A701009387070F93F7C7FF38
:106590002326F100973703009387C70D0327C10017
:1065A00023A0E700973703009387C70C23A20700B7
:1065B000973703009387870C379701001307C7FFAE
:1065C00023A2E700973703009387470B23A0070018
:1065D0008327C1002324F10083278100379701001E
:1065E0001307C7FF23A2E7008327810017370300A3
:1065F0001307C70823A0E7001300000013010101DF
:1066000067800000130101FE2326A1002324B100AE
:106610002322C10083278100232EF1008327C1009C
:10662000232CF1000327C10083278100B367F70003
:1066300093F73700639607066F00C0028327C101F6
:1066400003A707008327810123A0E7008327810197
:1066500093874700232CF1008327C10193874700CC
:10666000232EF100832741009387D7FF0327C10022
:10667000B307F70003278101E362F7FC6F004002D4
:106680000327C10193071700232EF10083278101FF
:1066900093861700232CD100034707002380E700CF
:1066A0000327C10083274100B307F70003278101B7
:1066B000E368F7FC8327C10013850700130101027B
:1066C00067800000130101FE2326A1002324B100EE
:1066D0002322C1000327C10083274100B367F700CD
:1066E00093F73700639807068327810093F7F70F26
:1066F000232AF10083274101939787000327410153
:10670000B367F700232AF10083274101939707011C
:1067100003274101B367F700232AF1008327C10053
:10672000232EF1006F0080018327C10113874700EA
:10673000232EE1000327410123A0E7000327C10026
:1067400083274100B307F7000327C101E36EF7FC7D
:106750006F00C0038327C100232CF1006F00C0012C
:106760008327810113871700232CE1000327810071
:106770001377F70F2380E7000327C1008327410029
:10678000B307F70003278101E36CF7FC8327C100FF
:10679000138507001301010267800000130101FE49
:1067A0002326A1008327C100232EF1006F000001E2
:1067B0008327C10193871700232EF1008327C1018E
:1067C00083C70700E39607FE0327C1018327C100A3
:1067D000B307F7401385070013010102678000002B
:1067E000130101FE2326A1002324B1008327C10049
:1067F000138717002326E10083C70700A30FF100CA
:1068000083278100138717002324E10083C7070033
:10681000230FF1008347F101638807000347F1016B
:106820008347E101E304F7FC0347F1018347E101FA
:10683000B307F740138507001301010267800000CA
:10684000130101FE2326A1002324B1008327C100E8
:10685000232EF10013000000032781009307170087
:106860002324F1008327C10193861700232ED10032
:10687000034707002380E70083C70700E39E07FC68
:106880008327C10013850700130101026780000000
:10689000130101FE2326A100232E0100232C010059
:1068A0006F0000018327C100938717002326F100A2
:1068B0008327C10003C7070093070002E304F7FE24
:1068C0008327C10003C707009307D002630AF700BC
:1068D0008327C10003C707009307B0026312F706BE
:1068E0008327C10083C70700938737FD93B717003D
:1068F00093F7F70F232CF1008327C100938717002C
:106900002326F1006F00C0030327C101930707008E
:1069100093972700B387E70093971700232EF10082
:106920008327C100138717002326E10083C70700D0
:10693000938707FD0327C101B307F700232EF1005A
:106940008327C10083C70700E39007FC83278101E9
:10695000638807008327C101B307F0406F00800000
:106960008327C1011385070013010102678000001E
:10697000130101FE2326A10097370300938787D4D4
:1069800083A707009386170017370300130787D3E1
:106990002320D7000327C1001377F70F9736030092
:1069A000938646D6B387F6002380E7000327C1000D
:1069B0009307A000630CF70097370300938787D0F5
:1069C00003A7070093070004631EF704973703002B
:1069D000938747D3232EF1006F00C0038327C101A3
:1069E00013871700232EE10003C70700B70710F035
:1069F000938707F023A0E70097370300938787CC9E
:106A000083A707001387F7FF97370300938787CB88
:106A100023A0E700973703009387C7CA83A707001F
:106A2000E39E07FA93070000138507001301010294
:106A300067800000130101EB232611142324811425
:106A40002322911423202115232E3113232C4113AB
:106A5000232A5113232EA100232CB1002328C10087
:106A6000232AD1002326E1002324F100232201015F
:106A7000232601128327C100138A0700930A00000E
:106A8000832701010328410113060A0093860A00A7
:106A90001385070093050800EF20005393070500B6
:106AA0001388050013860700930608008327C11288
:106AB000138717002326E112130706009397270078
:106AC00093060113B387F60023AEE7EE8327C100D8
:106AD00013840700930400008327410113870400F7
:106AE00063E8E70483274101138704006398E70004
:106AF000832701011307040063ECE7028327C10029
:106B00001389070093090000130609009386090002
:106B10000325010183254101EF10506D9307050006
:106B2000138805002328F100232A01016FF09FF448
:106B3000130000006F0040018327C10183258101FC
:106B400003254100E7800700832781001387F7FFB3
:106B50002324E1000327C112E340F7FE6F00400544
:106B60008327C1129397270013070113B307F70078
:106B700003A7C7EF8327C11293972700930601133A
:106B8000B387F60083A6C7EF9307900063F6D7009C
:106B9000930770056F00800093070003B387E70039
:106BA0000327C1018325810113850700E700070042
:106BB0008327C1121387F7FF2326E112E342F0FA7D
:106BC000130000008320C114032481148324411482
:106BD000032901148329C113032A8113832A411332
:106BE0001301011567800000130101FF2326A10096
:106BF0002324B10083268100130710006356D702B7
:106C00008327C10083A707009387770093F787FF47
:106C1000938687000327C1002320D70003A84700DD
:106C200083A707006F0000050327810063040702A4
:106C30000327C10003270700130647008326C1006E
:106C400023A0C600032707009307070013080000CE
:106C50006F0040020327C100032707001306470007
:106C60008326C10023A0C60003270700930707005F
:106C700013080000138507009305080013010101A4
:106C800067800000130101FF2326A1002324B10027
:106C900083268100130710006356D7028327C100A3
:106CA00083A707009387770093F787FF9386870072
:106CB0000327C1002320D70003A8470083A70700AC
:106CC0006F00800503278100630607020327C100C8
:106CD00003270700130647008326C10023A0C60030
:106CE00003270700930707001357F741130807000E
:106CF0006F0080020327C100032707001306470027
:106D00008326C10023A0C6000327070093070700BE
:106D10001357F74113080700138507009305080070
:106D20001301010167800000130101FC232E1102F1
:106D3000232C8102232A91022326A1002324B100BF
:106D40002322C1002320D1006F0040026300043CD5
:106D500083274100938717002322F1008327C10076
:106D60008325810013050400E78007008327410085
:106D700083C707001384070093075002E318F4FC4D
:106D800083274100938717002322F10083274100C6
:106D90002328F10093070002A30BF1009307F0FFF3
:106DA000232EF1009307F0FF232CF1002320010292
:106DB00083274100138717002322E10083C70700C0
:106DC000138407009307D4FD130750056360F7325F
:106DD00013972700979701009387C729B307F700F8
:106DE00003A70700979701009387C728B307F70009
:106DF000678007009307D002A30BF1006FF05FFBE1
:106E000093070003A30BF1006FF09FFA232C0100FE
:106E1000032781019307070093972700B387E700B3
:106E200093971700B307F400938707FD232CF10015
:106E30008327410083C70700138407009307F002EC
:106E400063D287049307900363CE870283274100B0
:106E5000938717002322F1006FF09FFB8327010027
:106E6000138747002320E10083A70700232CF100AC
:106E70006F0080018327C101E3DC07F2232E0100AC
:106E80006FF01FF3130000008327C101E3D207F264
:106E900083278101232EF1009307F0FF232CF100BB
:106EA0006FF01FF183270102938717002320F1025F
:106EB0006FF01FF083270100138747002320E100B4
:106EC00083A707000327C1008325810013850700DE
:106ED000E70007006F004023832701001387470066
:106EE0002320E10083A40700639604009794010027
:106EF0009384C4178327C1016350F00803477101CD
:106F00009307D002630AF706832781019385070060
:106F100013850400EF10502B130705008327C101D0
:106F2000B387E740232EF1006F00400283477101D1
:106F30000327C1008325810013850700E7000700B0
:106F40008327C1019387F7FF232EF1008327C10117
:106F5000E34EF0FC6F0040028327C10083258100CF
:106F600013050400E7800700938414008327C10100
:106F70009387F7FF232EF10083C7040013840700D3
:106F80006300040483278101E3C807FC8327810190
:106F90009387F7FF232CF10083278101E3DE07FAB3
:106FA0006F0000028327C1008325810013050002C2
:106FB000E78007008327C1019387F7FF232EF100A5
:106FC0008327C101E340F0FE6F0000149307010026
:106FD0008325010213850700EFF0DFCA9307050040
:106FE000138805002324F10223260103832781024D
:106FF0000328C1029307080063D607048327C10052
:10700000832581001305D002E780070083258102D4
:107010000326C1029307000013080000B386B7409F
:107020001385060033B5A7003307C840B307A74050
:107030001387070093870600130807002324F10233
:10704000232601039307A0002322F1026F004006CC
:107050009307A0002322F1026F0000049307800031
:107060002322F1026F004003930710002320F10256
:107070008327C1008325810013050003E7800700F3
:107080008327C1008325810013058007E78007005F
:10709000930700012322F1029307010083250102D7
:1070A00013850700EFF05FB42324A1022326B10269
:1070B0000327410283477101138807008327C10119
:1070C000032681028326C102832581000325C10096
:1070D000EFF05F966F0040038327C1008325810096
:1070E00013050400E78007006F0000028327C1003A
:1070F0008325810013055002E780070083270101E3
:107100002322F100130000006FF05FC6130000009F
:107110008320C10303248103832441031301010459
:1071200067800000130101FF2326A100B70710F0BC
:10713000938707F20327C10023A0E7006F00000038
:10714000130101FB232611022326A100232AB102E9
:10715000232CC102232ED1022320E1042322F10497
:10716000232401052326110593070105938747FE74
:10717000232EF1008327C101938607000326C10057
:107180009305000017F5FFFF1305C57EEFF0DFB98B
:1071900093070000138507008320C1021301010536
:1071A00067800000130101FE2326A1002324B10003
:1071B0002322710083278100232EF1008327C10140
:1071C00083A707000327C1001377F70F2380E70089
:1071D0008327C10183A70700138717008327C101F5
:1071E00023A0E700130000001301010267800000E4
:1071F000130101FA232E11022326A1002324B1003A
:107200002324C1042326D1042328E104232AF104E2
:10721000232C0105232E1105930701062322F102D9
:107220009307410193054101170600001306C6F7B5
:1072300037F7FFFF9346F7FF37150000130505806A
:107240003388A5003378E8001368783B23A0070152
:107250003305A6003377E5001367773323A2E700F1
:1072600033F7D500931547013787030013073739E4
:1072700033E7E50023A4E7003377D60093164701F0
:10728000370703001307770633E7E60023A6E70076
:107290000F1000008327C1002326F1029307010687
:1072A000938787FE2324F10203278102930741017C
:1072B000138507009307C10093060700032681008A
:1072C00093850700EFF05FA68327C10023800700A6
:1072D0008327C100138707008327C102B307F74044
:1072E000138507008320C103130101066780000096
:1072F000130101FF370510F0130545F403250500C0
:107300002326A100370510F0130505F40325050019
:107310002324A100370510F0130545F403250500CB
:107320008328C100E398A8FC0325C10013030500CE
:107330009303000013170300930600000325810048
:107340009305050013060000B3E7B6003368C700D5
:10735000370710F0130587F4B715000093858538BB
:1073600013060000B386B70093880600B3B8F80090
:107370003307C800B387E800138707009387060028
:10738000130807002320F500232205011300000045
:107390001301010167800000130101FF2326110082
:1073A000EFF01FF59307000873A0473013000000AB
:1073B0008320C1001301010167800000130101FE59
:1073C000232E11002326A10017950100130505E0C7
:1073D000EFF01FD7130000008320C1011301010249
:1073E00067800000130101FE232E11002326A10057
:1073F00017950100130505DEEFF09FD41300000080
:107400008320C1011301010267800000130101FD07
:10741000232611022326A100232E01006F00400124
:10742000130000008327C10193871700232EF1006A
:107430000327C101B717000093877738E3D2E7FE2F
:1074400017950100130585D9EFF09FCF6FF0DFFC92
:10745000130101FF23261100EF004022EF00102B43
:10746000EF00D070130000008320C1001301010160
:1074700067800000130101FE232E11002326010066
:10748000EF00901E1307050093071000630EF7002E
:1074900017950100130505D5EFF09FCA8327C1009A
:1074A00093E727002326F100EF00D06113070500C2
:1074B00093071000630EF700179501001305C5D45C
:1074C000EFF01FC88327C10093E747002326F10090
:1074D000EF10803E1307050093071000630EF700BE
:1074E000179501001305C5D4EFF09FC58327C10090
:1074F00093E787002326F1008327C1001385070047
:107500008320C1011301010267800000130101FE05
:10751000232E110023260100EFF09FF31707000030
:107520001307870693060000130610009305400614
:1075300017950100130505D2EFD05FB42326A100F3
:107540008327C10063820702EFB01F9A93070500EB
:107550001307000093060000138607009305100030
:107560000325C100EFD0DFBC23240100EFB0CFEA38
:1075700093070000138507008320C1011301010256
:1075800067800000130101FD232611022326A100BC
:1075900097970100938747F083A707001387470653
:1075A00097970100938747EF23A0E7009797010083
:1075B0009387C7EE83A707001387470697970100B5
:1075C0009387C7ED23A0E700979701009387C7EC47
:1075D00003A70700B7170000938777BB63D2E706BE
:1075E00097970100938747EB03A70700B7F7FFFFC3
:1075F000938787443307F700979701009387C7E97C
:1076000023A0E700EFF01FE7232EA1008327C1018D
:10761000639E070097970100938747E803A7070039
:10762000B72700009387773263D0E7028327C10131
:1076300013850700EFF01FAFEFB00FE96F000001F7
:10764000130000006F008000130000008320C102BF
:107650001301010367800000737004306F000000A5
:107660001300000067800000130101FF2326A10022
:107670002324B100737004306F000000130101FF78
:107680002326110013060000930540001305500047
:10769000EF90CFCC13070500972703009387870A45
:1076A00023A0E700972703009387C70983A7070054
:1076B000979501009385C5BA13850700EFA04FEF9A
:1076C0009308000013080000930700001307200030
:1076D000930600001306004097950100938585B935
:1076E000170500001305C504EFA09F85930800004F
:1076F000130800009727030093870705130710005E
:10770000930600001306004097950100938505B786
:10771000170500001305855BEFA09F821300000092
:107720008320C1001301010167800000130101FCE7
:10773000232E11022326A100232001026F00400BFB
:10774000832701021307A000B317F7002326F102D5
:10775000EFB08FF92324A10297270300938787FEB8
:1077600083A707001307C101930600000326C10287
:107770009305070013850700EF909FC3930705004B
:10778000638A0700972703009387C7FC130710003D
:1077900023A0E700EFB04FF5130705008327810210
:1077A000B307F7402322F102032741028327C102D6
:1077B000637AF700972703009387C7F91307100030
:1077C00023A0E7008327C1029387F7000327410224
:1077D00063FAE700972703009387C7F713071000A2
:1077E00023A0E70083270102938717002320F102DB
:1077F0000327010293074000E3D4E7F423200102AA
:107800006F000005972703009387C7F383A707003E
:1078100013070102930600001306000093050700FA
:1078200013850700EF900FEC130705009307100076
:10783000630AF700972703009387C7F11307100027
:1078400023A0E70083270102938717002320F1027A
:107850000327010293074000E3D6E7FA2320010241
:107860006F00400B832701021307A000B317F70036
:107870002326F102EFB04FE72324A102972703004C
:10788000938747EC83A707001307010293060000C4
:107890000326C1029305070013850700EF908FE4CC
:1078A00093070500638A070097270300938787EAF9
:1078B0001307100023A0E700EFB00FE31307050044
:1078C00083278102B307F7402322F10203274102F5
:1078D0008327C102637AF70097270300938787E71E
:1078E0001307100023A0E7008327C1029387F70046
:1078F0000327410263FAE70097270300938787E590
:107900001307100023A0E7008327010293871700C5
:107910002320F1020327010293074000E3D4E7F498
:1079200097270300938747E323A0070097270300C7
:10793000938787E183A7070013850700EFB00F8BBC
:107940006F00C00013054001EFA09FAB9727030015
:10795000938787E003A7070093075005E314F7FE1A
:1079600013054001EFA0DFA9972703009387C7DE27
:1079700023A00700232001026F0080109727030037
:10798000938747DC83A707001307C1019306000014
:10799000130600009305070013850700EF905FA111
:1079A0001307050093071000630AF70097270300E9
:1079B000938747DA1307100023A0E70097270300F7
:1079C000938747D883A70700130701029306000097
:1079D000130600009305070013850700EF908FD072
:1079E0001307050093071000630AF70097270300A9
:1079F000938747D61307100023A0E70097270300BB
:107A0000938787D503A7070093075005631AF700EC
:107A100097270300938707D41307100023A0E700DC
:107A200097270300938747D283A707009305400059
:107A300013850700EFA09FC0972703009387C7D146
:107A400003A7070093075005631AF7009727030061
:107A5000938747D01307100023A0E7009727030060
:107A6000938787CE83A7070093051000138507002F
:107A7000EFA0DFBC83270102938717002320F102C8
:107A80000327010293074000E3DAE7EE6F00C0002E
:107A900013054001EFA0DF96972703009387C7CB1C
:107AA00003A7070093075005E314F7FE13054001F1
:107AB000EFA01F9597270300938707CA23A007000D
:107AC000232001026F00000597270300938787C7D3
:107AD00083A707001307C1019306000013060000E7
:107AE0009305070013850700EF909F8C130705008F
:107AF00093071000630AF70097270300938787C551
:107B00001307100023A0E7008327010293871700C3
:107B10002320F1020327010293074000E3D6E7FA8E
:107B200097270300938747C283A7070013850700A1
:107B3000EFA0DFEB6F00C00013054001EFA05F8CEA
:107B400097270300938747C103A7070093075005B2
:107B5000E314F7FE13054001EFA09F8A9727030067
:107B6000938787BF23A00700232001026F008010A6
:107B700097270300938707BD83A707001307010218
:107B80009306000013060000930507001385070005
:107B9000EF904FB51307050093071000630AF70035
:107BA00097270300938707BB1307100023A0E70064
:107BB00097270300938707B983A707001307C1011D
:107BC00093060000130600009305070013850700C5
:107BD000EF900FFE1307050093071000630AF700EC
:107BE00097270300938707B71307100023A0E70028
:107BF00097270300938747B603A70700930750050D
:107C0000631AF700972703009387C7B41307100080
:107C100023A0E70097270300938707B383A70700F4
:107C20009305400013850700EFA05FA1972703008D
:107C3000938787B203A7070093075005631AF700DD
:107C400097270300938707B11307100023A0E700CD
:107C500097270300938747AF83A70700930510007A
:107C600013850700EFA09F9D8327010293871700CC
:107C70002320F1020327010293074000E3DAE7EE35
:107C80006F00C00013054001EFA08FF79727030096
:107C9000938787AC03A7070093075005E314F7FE0B
:107CA00013054001EFA0CFF597270300938707AA9C
:107CB00083A707001387170097270300938707A957
:107CC00023A0E7006FF05FA7130101FD2326110237
:107CD0002326A10013050000EFA09FB6EFB0CFA0B0
:107CE000232EA100232A0100972703009387C7A60C
:107CF0001307500523A0E70097270300938787A465
:107D000083A7070013074101930600001306F00A3A
:107D10009305070013850700EF90CF9C930705009C
:107D2000638A0700972703009387C7A213071000F1
:107D300023A0E700EFB04F9B130705008327C10185
:107D4000B307F740232CF100032781019307E00AD2
:107D500063EAE700972703009387C79F1307100084
:107D600023A0E700032781019307E00B63FAE700F4
:107D7000972703009387079E1307100023A0E700AF
:107D8000972703009387479D1307500523A0E7001B
:107D900013050000EFA0DFAAEFB00F95232EA1007E
:107DA000972703009387479B1307500523A0E700FD
:107DB000972703009387079983A7070013074101BB
:107DC000930600001306F00A9305070013850700C9
:107DD000EF900FDE93070500638A070097270300E3
:107DE000938747971307100023A0E700EFB0CF8FCA
:107DF000130705008327C101B307F740232CF100C7
:107E0000032781019307E00A63EAE700972703004D
:107E1000938747941307100023A0E70003278101ED
:107E20009307E00B63FAE700972703009387879295
:107E30001307100023A0E700972703009387C7913B
:107E40001307500523A0E700972703009387479067
:107E500083A7070013871700972703009387478F8F
:107E600023A0E7006FF01FE7130101FF9307100045
:107E70002326F100972703009387478D03A7070068
:107E8000972703009387878D83A707006314F70064
:107E900023260100972703009387878B03A70700FA
:107EA000972703009387C78B83A707006314F70006
:107EB00023260100972703009387C78903A707009C
:107EC000930710006314F70023260100972703008F
:107ED0009387078803A7070097270300938747889E
:107EE00023A0E700972703009387478603A707008F
:107EF000972703009387878623A0E7008327C10085
:107F0000138507001301010167800000130101FFC1
:107F1000232611009305800C1305800CEF809FF43D
:107F200013070500972703009387078423A0E70022
:107F300097270300938747831307A00A23A2E7002C
:107F4000972703009387478223A407009305000027
:107F50001305800CEF801FF113070500972703001E
:107F60009387878023A6E700971703009387C77F2F
:107F700023A80700971703009387077F23AA07000A
:107F8000971703009387477E83A707009785010013
:107F90009385452F13850700EF909FE19717030006
:107FA0009387877C83A7C700978501009385852EDB
:107FB00013850700EF90DFDF971703009387C77AD9
:107FC00083A70700639A0700971703009387C77971
:107FD00083A7C70063820706930800001308000008
:107FE0009307000013070000971603009386C677D7
:107FF00013060040978501009385C52A17050000E8
:1080000013054521EF90DFF39308000013080000EB
:1080100093070000130700009716030093868675E8
:108020001306004097850100938545281705000039
:108030001305451EEF90DFF0130000008320C10000
:108040001301010167800000130101FD23261102C5
:108050002326A1002324B10093060000130600008C
:10806000930500000325C100EF80DFE7130705003B
:1080700093071000631AF700971703009387876E22
:108080001307100023A0E700232E01006F00400516
:108090009306000013060000930500000325C100AD
:1080A000EF900FB11307050093071000630AF70064
:1080B000971703009387076B1307100023A0E700AF
:1080C0008327810083A70700138717008327810078
:1080D00023A0E7008327C10193871700232EF10017
:1080E0000327C1019307700CE3F4E7FA930600003D
:1080F00013060000930500000325C100EF904FAB6D
:108100001307050093071000631AF7009717030081
:10811000938747651307100023A0E70013000000B2
:108120008320C1021301010367800000130101FDD8
:10813000232611022326A1002324B1009306000068
:1081400013060000930500000325C100EF904FA621
:108150001307050093071000631AF7009717030031
:10816000938747601307100023A0E700232E010028
:108170006F00400593060000130600009305000001
:108180000325C100EF801FD61307050093071000D9
:10819000630AF700971703009387C75C1307100063
:1081A00023A0E7008327810083A707001387170018
:1081B0008327810023A0E7008327C101938717004D
:1081C000232EF1000327C1019307700CE3F4E7FAB3
:1081D0009306000013060000930500000325C1006C
:1081E000EF805FD01307050093071000631AF700B4
:1081F00097170300938707571307100023A0E70082
:10820000130000008320C1021301010367800000F6
:10821000130101FD232611022326A1008327C1009B
:10822000232EF1008327C10103A747009307A00A6B
:108230006310F7028327C10103A707008327C10149
:10824000938787009385070013050700EFF0DFDFB2
:108250008327C10183A707009306000013060000CF
:108260009305000013850700EF908F941307050016
:1082700093071000631AF700971703009387874E40
:108280001307100023A0E7008327C10103A70700FD
:108290008327C10193878700938507001305070093
:1082A000EFF0DFE88327C10103A707008327C1019F
:1082B000938787009385070013050700EFF0DFD849
:1082C0006FF09FFC130101FF930710002326F100BC
:1082D000971703009387074983A707006384070064
:1082E00023260100971703009387074803A78700F9
:1082F000971703009387C74883A707006316F70003
:10830000232601006F00C001971703009387C7451C
:1083100003A78700971703009387874623A0E700EA
:10832000971703009387474403A747019717030054
:108330009387474583A707006316F70023260100AC
:108340006F00C001971703009387074203A74701F7
:10835000971703009387074323A0E7008327C100F3
:10836000138507001301010167800000130101FF5D
:108370002326110013054000EF809F8D1307050091
:10838000971703009387474023A0E7009717030040
:108390009387873F83A7070097850100938585F121
:1083A00013850700EF90DFA0971703009387C73D61
:1083B00083A70700638807089308000013080000DC
:1083C000971703009387073E1307200093060000CA
:1083D00013060040978501009385C5EE1705000040
:1083E00013058507EF90DFB5930800001308000020
:1083F000971703009387473B13071000930600006D
:108400001306004097850100938545EC1705000091
:108410001305C51AEF90DFB293080000130800009F
:1084200093070000130700009306000013060040A6
:1084300097850100938505EA1705000013050529B6
:10844000EF901FB0130000008320C1001301010151
:1084500067800000130101FD232611022326A100DD
:10846000971703009387473283A7070013850700F8
:10847000EF80DF8A1307050093071000631AF700E7
:1084800097170300938787301307100023A0E70096
:10849000232E01006F00C004971703009387C72E97
:1084A00083A707009305800013850700EF809F9046
:1084B0001307050093071000630AF70097170300DE
:1084C0009387C72C1307100023A0E7001305400172
:1084D000EF901FF38327C10193871700232EF1002C
:1084E0000327C10193079000E3F8E7FA232E010068
:1084F0006F00800413054001EF909FF09717030071
:108500009387872883A7070013850700EF801F81C3
:108510001307050093071000630AF700971703007D
:108520009387C7261307100023A0E7008327C10104
:1085300093871700232EF1000327C10193079000B2
:10854000E3FAE7FA971703009387072483A7070046
:1085500013850700EF808FFC1307050093071000B9
:10856000631AF70097170300938747221307100039
:1085700023A0E700971703009387072283A707002C
:1085800013871700971703009387072123A0E7009D
:10859000971703009387C71F1307100023A0E70056
:1085A00013050000EFA0CFA9971703009387471E7C
:1085B00023A007006FF0DFEA130101FE232E110054
:1085C0002326A100971703009387071C83A70700A2
:1085D0009305E0FF13850700EF80CFFD130705002B
:1085E000930710006312F708971703009387471A41
:1085F00003A7070093071000630CF7009717030009
:108600009387C7181307100023A0E7006F00C00668
:10861000971703009387471783A707001385070061
:10862000EF80CFEF1307050093071000630AF700F0
:1086300097170300938787151307100023A0E700FF
:1086400097170300938707151307100023A0E7006F
:1086500013050000EFA0CF9E9717030093878713A1
:1086600023A007006F0040019717030093870712AC
:108670001307100023A0E700971703009387071242
:1086800083A7070013871700971703009387C71066
:1086900083A70700630AF700971703009387070F64
:1086A0001307100023A0E700971703009387070F15
:1086B00083A7070013871700971703009387070EF8
:1086C00023A0E7006FF01FF0130101FE232E11001D
:1086D0002326A100971703009387070B83A70700A2
:1086E0009305000013850700EF80CFEC130705000A
:1086F00093071000E310F7FE971703009387870A8C
:1087000083A7070013850700EF909FD81307050084
:10871000930730006306F700737004306F000000A9
:10872000971703009387470883A70700138507005F
:10873000EF901FD613070500930730006306F7007C
:10874000737004306F00000097170300938787044D
:1087500003A7070093071000631CF7009717030097
:108760009387070303A7070093071000630CF70024
:1087700097170300938787011307100023A0E700D2
:108780006F004013971703009387870183A70700A3
:1087900013871700971703009387870023A0E7002C
:1087A000971703009387470083A7070013850700E7
:1087B000EFA0CFA3971703009387C7FE83A70700F7
:1087C00013850700EFA08FA297170300938787FCFC
:1087D00003A7070093071000630CF7009717030027
:1087E000938707FB03A7070093071000631AF7009E
:1087F00097170300938787F91307100023A0E7005A
:1088000013050000EF901FD8130705009307200001
:108810006306F700737004306F00000097170300C1
:10882000938747F883A7070013850700EF905FC67B
:1088300013070500930720006306F70073700430E8
:108840006F00000097170300938707F683A70700C0
:1088500013850700EF90DFC313070500930720007F
:108860006306F700737004306F0000009717030071
:10887000938787F183A7070013850700EF800FCA4E
:108880001307050093071000630AF700971703000A
:108890009387C7EF1307100023A0E700130500001C
:1088A000EF905FCE93070500E38607E27370043014
:1088B0006F0000006FF01FE2130101FF9717030024
:1088C0009387C7EE03A70700971703009387C7ECAA
:1088D00083A70700631CF70097170300938707EB34
:1088E0001307100023A0E7006F00C00197170300D3
:1088F000938787EA03A7070097170300938707EB7F
:1089000023A0E70097170300938787EA03A70700D0
:1089100097170300938787E883A70700631CF70076
:1089200097170300938787E61307100023A0E7003B
:108930006F00C00197170300938747E603A707005E
:10894000971703009387C7E623A0E7009717030054
:10895000938747E603A7070097170300938747E429
:1089600083A70700631CF70097170300938707E2AC
:108970001307100023A0E7006F00C0019717030042
:10898000938707E203A7070097170300938787E2FF
:1089900023A0E70097170300938747DF03A707008B
:1089A000930710006316F700232601006F00C00034
:1089B000930710002326F1008327C10013850700C9
:1089C0001301010167800000B305B500930705009E
:1089D0006386B70003C70700631607003385A74007
:1089E00067800000938717006FF09FFE130101FD61
:1089F00023229102232A51012326110223248102DA
:108A000023202103232E3101232C4101232861013E
:108A10002326710123248101232291012320A10116
:108A2000930A050093840500639E0638130406002C
:108A300093090500178901001309498A63F8C512D3
:108A4000B7070100138B05006378F6101307F00FCA
:108A50003337C70013173700B357E6003309F9005F
:108A6000834609003387E60093060002B386E6409A
:108A7000638C0600B394D40033D7EA003314D600D5
:108A8000336B9700B399DA00935A040193850A0077
:108A900013050B00EF00902A1309050093850A00C7
:108AA000931B040113050B00EF00D02493DB0B0193
:108AB000930405009305050013850B00EF00D020FB
:108AC0001319090193D70901B367F900138A040048
:108AD00063FEA700B3878700138AF4FF63E887006B
:108AE00063F6A700138AE4FFB3878700B384A74027
:108AF00093850A0013850400EF0050241309050034
:108B000093850A0013850400EF00D01E9399090194
:108B100093040500930505001319090113850B0043
:108B200093D90901EF00501AB36939011386040083
:108B300063FCA900B30934011386F4FF63E68900DE
:108B400063F4A9001386E4FF13140A013364C4001C
:108B5000130A00006F000013B7070001130700019C
:108B6000E36CF6EE130780016FF01FEF138A060027
:108B7000631A06009305000013051000EF0090171C
:108B800013040500B7070100637EF4129307F00F8A
:108B900063F48700130A8000B35744013309F900D6
:108BA000034709009306000233074701B386E640F6
:108BB00063940612B3848440130A1000135B04010B
:108BC00093050B0013850400EF00501713090500EF
:108BD00093050B0013850400931B0401EF00901113
:108BE00093DB0B01930405009305050013850B002F
:108BF000EF00900D1319090193D70901B367F9002C
:108C0000938A040063FEA700B3878700938AF4FF6A
:108C100063E8870063F6A700938AE4FFB3878700C1
:108C2000B384A74093050B0013850400EF001011D7
:108C30001309050093050B0013850400EF00900B4A
:108C4000939909019304050093050500131909017F
:108C500013850B0093D90901EF001007B36939019F
:108C60001386040063FCA900B30934011386F4FFE2
:108C700063E6890063F4A9001386E4FF13940A01F4
:108C80003364C4001305040093050A008320C10265
:108C90000324810283244102032901028329C101A3
:108CA000032A8101832A4101032B0101832BC10087
:108CB000032C8100832C4100032D010013010103CB
:108CC00067800000B7070001130A0001E366F4ECB7
:108CD000130A80016FF05FEC3314D40033DAE40040
:108CE000B399DA0033D7EA00935A0401B394D4005D
:108CF00093850A0013050A00336B9700EF001004F8
:108D00001309050093850A0013050A00931B04014B
:108D1000EF00407E93DB0B019304050093050500F3
:108D200013850B00EF00407A1319090113570B014B
:108D30003367E900138A0400637EA70033078700C6
:108D4000138AF4FF636887006376A700138AE4FF41
:108D500033078700B304A74093850A0013850400F6
:108D6000EF00C07D1309050093850A0013850400F8
:108D7000EF004078930405009305050013850B0070
:108D8000EF00807413170B01135707011319090122
:108D9000B367E9001387040063FEA700B387870069
:108DA0001387F4FF63E8870063F6A7001387E4FFE7
:108DB000B3878700131A0A01B384A740336AEA0015
:108DC0006FF0DFDF63ECD51EB707010063F4F60434
:108DD0001307F00FB335D7009395350033D7B6009E
:108DE000977701009387874FB387E70003C7070092
:108DF000130A00023307B700330AEA4063160A0277
:108E000013041000E3E096E833B6CA0013441600DA
:108E10006FF05FE7B707000193050001E3E0F6FCA0
:108E2000930580016FF09FFBB35CE600B3964601AB
:108E3000B3ECDC0033D4E40093DB0C01B3974401C2
:108E400033D7EA0093850B0013050400336BF7005A
:108E5000B3194601EF00806E1309050093850B00DE
:108E600013050400139C0C01EF00C068135C0C0197
:108E7000930405009305050013050C00EF00C06482
:108E80001319090113570B013367E9001384040018
:108E9000637EA700330797011384F4FF636897018B
:108EA0006376A7001384E4FF33079701B304A74058
:108EB00093850B0013850400EF004068130905003B
:108EC00093850B0013850400EF00C0629304050036
:108ED0009305050013050C00EF00005F93170B01CD
:108EE0001319090193D70701B367F900138604002A
:108EF00063FEA700B38797011386F4FF63E8970129
:108F000063F6A7001386E4FFB387970113140401E7
:108F1000B70B01003364C4001389FBFF337D2401C8
:108F200033F92901B384A7409305090013050D0007
:108F3000EF008059935C040193050900130B0500B1
:108F400013850C00EF00405893D90901130C05005C
:108F50009385090013850C00EF00005713090500E5
:108F60009385090013050D00EF00005633058501B8
:108F700093570B013385A700637485013309790189
:108F800093570501B387270163E6F402E392F4BC2B
:108F9000B70701009387F7FF3375F5001315050137
:108FA000337BFB0033964A0133056501130A000049
:108FB000E37AA6CC1304F4FF6FF09FB9130A000004
:108FC000130400006FF01FCC130101FB2324810464
:108FD00023229104232E31032322910323261104FB
:108FE00023202105232C4103232A51032328610335
:108FF00023267103232481032320A103232EB101FF
:10900000930C050093890500130405009384050063
:10901000639E062613090600138A0600977A01004C
:10902000938ACA2B63F4C514B70701006376F6125E
:109030009307F00F63F4C700130A8000B35746018B
:10904000B38AFA0003C70A00130500023307470179
:10905000330AE540630C0A00B395490133D7EC00AD
:1090600033194601B364B70033944C01935A090194
:1090700093850A0013850400EF00404C9309050016
:1090800093850A00131B090113850400EF00804635
:10909000135B0B019305050013050B00EF00C042A5
:1090A0009399090193570401B3E7F90063FAA70004
:1090B000B387270163E6270163F4A700B38727017D
:1090C000B384A74093850A0013850400EF0000478E
:1090D0009309050093850A0013850400EF00804181
:1090E00013140401930505009399090113050B005E
:1090F00013540401EF00403D33E48900637AA40077
:1091000033042401636624016374A400330424013E
:109110003304A44033554401930500008320C10467
:109120000324810483244104032901048329C10306
:10913000032A8103832A4103032B0103832BC102EA
:10914000032C8102832C4102032D0102832DC101D6
:109150001301010567800000B7070001130A000131
:10916000E36EF6EC130A80016FF05FED631A060000
:109170009305000013051000EF00C0371309050028
:10918000B7070100637AF90E9307F00F63F4270124
:10919000130A8000B3574901B38AFA0003C70A00D3
:1091A00013050002B384294133074701330AE54020
:1091B000E30E0AEA33194901B3DAE900B39549012C
:1091C00033D7EC0093540901336BB70013850A00C1
:1091D00093850400EF008036930905009385040011
:1091E000931B090113850A00EF00C03093DB0B01CC
:1091F0009305050013850B00EF00002D93990901DD
:1092000093570B01B3E7F90033944C0163FAA700BD
:10921000B387270163E6270163F4A700B38727011B
:10922000B38AA7409385040013850A00EF0000313C
:10923000930905009385040013850A00EF00802B35
:109240009305050013850B00EF00002893150B0113
:109250009399090193D50501B3E5B90063FAA50017
:10926000B385250163E6250163F4A500B3852501D7
:10927000B384A5406FF09FDFB7070001130A000118
:10928000E36AF9F0130A80016FF0DFF0E3E8D5E854
:10929000B707010063FCF604930BF00F33B5DB0056
:1092A0001315350033D7A60097770100938707037E
:1092B000B387E70083CB070093050002B38BAB00B5
:1092C000338B7541631E0B0263E4360163EACC0005
:1092D0003384CC40B386D94033B58C00B384A640E8
:1092E00013050400938504006FF05FE3B7070001E6
:1092F00013050001E3E8F6FA130580016FF09FFA09
:10930000B3966601335D7601336DDD0033D47901A8
:10931000B395690133DC7C0193540D01336CBC00BF
:109320001305040093850400B31A6601EF000021C1
:10933000130A0500938504001305040033996C019A
:10934000931C0D01EF00001B93DC0C0113040500BE
:109350009305050013850C00EF000017131A0A018E
:1093600013570C013367EA00130A0400637EA70059
:109370003307A701130AF4FF6368A7016376A70008
:10938000130AE4FF3307A701B309A740938504003C
:1093900013850900EF00801A93850400130405006B
:1093A00013850900EF0000159305050093040500DF
:1093B00013850C00EF00401193150C0113140401E8
:1093C00093D50501B365B4001387040063FEA500BF
:1093D000B385A5011387F4FF63E8A50163F6A50033
:1093E0001387E4FFB385A501131A0A01B70C010026
:1093F000336AEA001384FCFFB3778A0033F48A00EF
:10940000B384A54013850700930504002326F100CB
:10941000135A0A01EF00400B93090500930504005D
:1094200013050A00EF00400A13DC0A01930D050042
:1094300093050C0013050A00EF0000098327C10003
:10944000130A050093050C0013850700EF00C00701
:109450003305B50113D709013307A7006374B701BA
:10946000330A9A01B70701009387F7FF9355070165
:109470003377F70013170701B3F7F900B3854501F8
:10948000B307F70063E6B400639EB400637CF900A1
:1094900033865741B3B7C700B385A541B385F540BF
:1094A00093070600B307F9403339F900B385B44098
:1094B000B385254133947501B3D767013365F40053
:1094C000B3D565016FF09FC51306050013050000B5
:1094D00093F61500638406003305C50093D5150087
:1094E00013161600E39605FE67800000634005062C
:1094F00063C6050613860500930505001305F0FFF6
:10950000630C060293061000637AB6006358C0002D
:109510001316160093961600E36AB6FE13050000B4
:1095200063E6C500B385C5403365D50093D6160004
:1095300013561600E39606FE678000009382000033
:10954000EFF05FFB13850500678002003305A04044
:1095500063D80500B305B0406FF0DFF9B305B04044
:1095600093820000EFF01FF93305A04067800200EE
:109570009382000063CA0500634C0500EFF09FF77B
:109580001385050067800200B305B040E35805FE6F
:109590003305A040EFF01FF63305B04067800200AE
:02000004800278
:1000000049444C4500000000244BFEFFBC4AFEFF63
:10001000D84AFEFFF04AFEFF004BFEFFF44CFEFF05
:100020008C4CFEFFA84CFEFFC04CFEFFD04CFEFFE8
:10003000546D7220537663001C56FEFF1C56FEFF63
:100040001C56FEFF0457FEFFAC56FEFFF456FEFFA3
:100050001C56FEFF1C56FEFF0457FEFFAC56FEFF6B
:10006000546D725100000000286E756C6C29000000
:10007000406DFEFF7C70FEFF6870FEFF7C70FEFF2F
:100080007C70FEFF7C70FEFF7C70FEFFEC6DFEFF5F
:100090007C70FEFF7C70FEFF846DFEFF046EFEFF31
:1000A0007C70FEFF906DFEFF9C6DFEFF9C6DFEFF61
:1000B0009C6DFEFF9C6DFEFF9C6DFEFF9C6DFEFF28
:1000C0009C6DFEFF9C6DFEFF9C6DFEFF7C70FEFF35
:1000D0007C70FEFF7C70FEFF7C70FEFF7C70FEFF7C
:1000E0007C70FEFF7C70FEFF7C70FEFF7C70FEFF6C
:1000F0007C70FEFF7C70FEFF7C70FEFF7C70FEFF5C
:100100007C70FEFF7C70FEFF7C70FEFF7C70FEFF4B
:100110007C70FEFF7C70FEFF7C70FEFF7C70FEFF3B
:100120007C70FEFF7C70FEFF7C70FEFF7C70FEFF2B
:100130007C70FEFF7C70FEFF7C70FEFF7C70FEFF1B
:100140007C70FEFF7C70FEFF7C70FEFF7C70FEFF0B
:100150007C70FEFF7C70FEFF7C70FEFF7C70FEFFFB
:100160007C70FEFF7C70FEFF7C70FEFF7C70FEFFEB
:10017000446EFEFF5C6FFEFF7C70FEFF7C70FEFF36
:100180007C70FEFF7C70FEFF7C70FEFF7C70FEFFCB
:100190007C70FEFF346EFEFF7C70FEFF7C70FEFF05
:1001A000EC6FFEFFF86FFEFF7C70FEFF7C70FEFFC1
:1001B000686EFEFF7C70FEFFE06FFEFF7C70FEFF4E
:1001C0007C70FEFF2070FEFF6D69616F750A000094
:1001D0006D69616F75320A0068756E6772790A0021
:1001E0004572726F7220696E20626C6F636B20744F
:1001F000696D652074657374207461736B73200D71
:100200000A0000004572726F7220696E20636F757C
:100210006E74696E672073656D6170686F726520BA
:100220007461736B73200D0A000000004572726FD9
:100230007220696E20726563757273697665206DD0
:1002400075746578207461736B73200D0A0000006B
:10025000436865636B54696D65720000426C6F633F
:100260006B5F54696D655F517565756500000000D1
:100270004254657374310000425465737432000057
:10028000436F756E74696E675F53656D5F31000013
:10029000436F756E74696E675F53656D5F32000002
:1002A000434E543100000000434E54320000000021
:1002B0005265637572736976655F4D757465780014
:1002C0005265633100000000526563320000000097
:1002D00052656333000000000001020203030303C0
:1002E00004040404040404040505050505050505C6
:1002F00005050505050505050606060606060606A6
:10030000060606060606060606060606060606068D
:100310000606060606060606070707070707070775
:10032000070707070707070707070707070707075D
:10033000070707070707070707070707070707074D
:10034000070707070707070707070707070707073D
:100350000707070707070707080808080808080825
:10036000080808080808080808080808080808080D
:1003700008080808080808080808080808080808FD
:1003800008080808080808080808080808080808ED
:1003900008080808080808080808080808080808DD
:1003A00008080808080808080808080808080808CD
:1003B00008080808080808080808080808080808BD
:1003C00008080808080808080808080808080808AD
:0803D0000808080808080808E5
:1003D8001000000000000000017A5200017C0101B9
:1003E8001B0D02004C00000018000000F885FEFFFD
:1003F800DC05000000440E307089039507810188F0
:100408000292049305940696089709980A990B9AFC
:100418000C0370020AC144C844C944D244D344D42A
:1004280044D544D644D744D844D944DA440E004489
:100438000B0000005000000068000000848BFEFFE5
:100448000005000000440E50748802890393059942
:100458000B810192049406950796089709980A9AC1
:100468000C9B0D0320010AC144C844C944D244D39B
:1004780044D444D544D644D744D844D944DA44DB98
:08048800440E00440B000000CB
:10049C00AAAAAAAA08000000FC8F01000400000010
:040000058000004037
:00000001FF
